:0300000002699101
:10699100758E1190000078FF79FFE4F0A3D9FBD840
:0D69A100F778FFE4F6D8FD75817F0269E903
:106D84004401EA40490FDB4401E640C90FDB4401FA
:056D9400E23C8EFA351F
:064A40009001CA122028BB
:104A46009001CEE0FCA3E0FDA3E0FEA3E0FFEF248F
:104A560069FFEE3474FEED34FFFDEC34FFFCEC121E
:104A66001B927BDF7A927986783D12196E9001D27D
:104A76001220287B007A0079C078419001D2E0FCB0
:104A8600A3E0FDA3E0FEA3E0FF121A771261FD7B0F
:104A9600007A0079C0784112196EC004C005C006BC
:104AA600C0077F977E7E7DD57C409001D2E0F8A33B
:104AB600E0F9A3E0FAA3E0FB12187DD003D002D000
:104AC60001D000121879C004C005C006C0077F9245
:104AD6007E867DC07C419001CAE0F8A3E0F9A3E0A0
:104AE600FAA3E0FB12196EA804A905AA06AB07D023
:104AF60007D006D005D00412187D9001DA122028BE
:104B06009001CEE0FCA3E0FDA3E0FEA3E0FFEF24CE
:104B160069FFEE3474FEED34FFFDEC34FFFCEC125D
:104B26001B929001CAE0F8A3E0F9A3E0FAA3E0FB28
:104B360012187D7B307AE67958783D12196EA804F2
:104B4600A905AA06AB077F817E0E7DBA7C431218A3
:104B5600799001E2E0F8A3E0F9A3E0FAA3E0FB1202
:104B6600196E9001D61220289001E6E0FCA3E0FD24
:104B7600A3E0FEA3E0FF9001D6E0F8A3E0F9A3E0EE
:104B8600FAA3E0FB121B14602940279001D6E0FC33
:104B9600A3E0FDA3E0FEA3E0FF9001E6E0F8A3E0BA
:104BA600F9A3E0FAA3E0FB1218799001D6122028A7
:104BB60080B69001E6E0FCA3E0FDA3E0FEA3E0FFE3
:104BC600121B819001D6E0F8A3E0F9A3E0FAA3E076
:104BD600FB121B1450279001D6E0FCA3E0FDA3E0D6
:104BE600FEA3E0FF9001E6E0F8A3E0F9A3E0FAA354
:104BF600E0FB12187D9001D612202880B57F007E3A
:104C0600007D007C009001D6E0F8A3E0F9A3E0FA6D
:104C1600A3E0FB121B14604840469001EAE0FCA3A7
:104C2600E0FDA3E0FEA3E0FF9001D6E0F8A3E0F9E3
:104C3600A3E0FAA3E0FB121B1450259001D6E0FC7A
:104C4600A3E0FDA3E0FEA3E0FF9001E6E0F8A3E009
:104C5600F9A3E0FAA3E0FB1218799001D6122028F6
:104C66007F007E007D007C009001D6E0F8A3E0F98D
:104C7600A3E0FAA3E0FB121B14504B9001EAE0FC00
:104C8600A3E0FDA3E0FEA3E0FF121B819001D6E0A6
:104C9600F8A3E0F9A3E0FAA3E0FB121B1460274097
:104CA600259001D6E0FCA3E0FDA3E0FEA3E0FF9083
:104CB60001E6E0F8A3E0F9A3E0FAA3E0FB12187D11
:104CC6009001D61220289001D6E0FCA3E0FDA3E0D7
:104CD600FEA3E0FF125A637B247A0B799878391287
:104CE600196E9001DAE0F8A3E0F9A3E0FAA3E0FB7D
:104CF60012187D9001DE1220287B007A0079C07898
:104D0600419001DEE0FCA3E0FDA3E0FEA3E0FF127C
:104D16001A771261FD7B007A0079C0784112196E0C
:104D2600A804A905AA06AB079001DEE0FCA3E0FDF6
:094D3600A3E0FEA3E0FF121879CE
:014D3F002251
:106E11009001F51220289001F5E0FCA3E0FDA3E02C
:106E2100FEA3E0FF1261FDA804A905AA06AB079025
:106E310001F5E0FCA3E0FDA3E0FEA3E0FF12187959
:106E41009001E6E0F8A3E0F9A3E0FAA3E0FB121950
:026E51006E22AF
:060D470090015A12202861
:100D4D0090015AE0FCA3E0FDA3E0FEA3E0FFEF2439
:100D5D0013FFEE342DFEED34FFFDEC34FFFCEC12F1
:100D6D001B9290015EE0F8A3E0F9A3E0FAA3E0FB8B
:100D7D0012187D9001621220287F8D7EA67D147C35
:100D8D003D900162E0F8A3E0F9A3E0FAA3E0FB12C5
:100D9D00196E7B807AF279BF783E12187D126E1132
:100DAD009001661220287F477E857D167C3D90013F
:100DBD0062E0F8A3E0F9A3E0FAA3E0FB12196E7B61
:100DCD00937AA77984783E12187D126E1190016A7C
:100DDD001220287F217EB47D0A7C3D900162E0F8CF
:100DED00A3E0F9A3E0FAA3E0FB12196E7BFF7ACD25
:100DFD007953783F12187D126E1190016E122028D2
:100E0D007F4D7E6C7D337C3B900162E0F8A3E0F971
:100E1D00A3E0FAA3E0FB12196E7B817A3D797E780F
:100E2D003F12187D126E119001721220287F007EE4
:100E3D00007D007C4090016EE0F8A3E0F9A3E0FA9C
:100E4D00A3E0FB12196EA804A905AA06AB07900131
:100E5D0066E0FCA3E0FDA3E0FEA3E0FF121879120B
:100E6D005A4D7BF37A767914783F12196EC004C00F
:100E7D0005C006C007900166E0FCA3E0FDA3E0FEFF
:100E8D00A3E0FF125A4D7BE87AC1795178401219CF
:100E9D006EA804A905AA06AB077FB17E737D717C90
:100EAD0042121879D003D002D001D000121879C0A7
:100EBD0004C005C006C0077F007E007D007C409009
:100ECD00016EE0F8A3E0F9A3E0FAA3E0FB12196EBE
:100EDD00125A4D7B0C7A5979ED783E12196EA80491
:100EED00A905AA06AB07D007D006D005D004121865
:100EFD00799001761220287F007E007D007C409045
:100F0D00016EE0F8A3E0F9A3E0FAA3E0FB12196E7D
:100F1D00C004C005C006C0077F007E007D007C4078
:100F2D00900166E0F8A3E0F9A3E0FAA3E0FB121943
:100F3D006ED003D002D001D000121879125A4D7B19
:100F4D00767A4F791E783D12196EC004C005C00621
:100F5D00C0077F007E007D007C40900166E0F8A315
:100F6D00E0F9A3E0FAA3E0FB12196E125A4D7B9C37
:100F7D007A5A79B6783D12196EA804A905AA06AB5E
:100F8D0007900176E0FCA3E0FDA3E0FEA3E0FF12D5
:100F9D001879A804A905AA06AB07D007D006D00575
:100FAD00D00412187DC004C005C006C0077F007EA6
:100FBD00007D007C4090016EE0F8A3E0F9A3E0FA1B
:100FCD00A3E0FB12196E900172E0F8A3E0F9A3E023
:100FDD00FAA3E0FB121879125A4D7B687A967904C0
:100FED00783D12196EA804A905AA06AB07D007D043
:100FFD0006D005D0041218799001761220287F00B2
:10100D007E007D007C4090016EE0F8A3E0F9A3E046
:10101D00FAA3E0FB12196EA804A905AA06AB079066
:10102D000166E0FCA3E0FDA3E0FEA3E0FF1218794A
:10103D00900172E0F8A3E0F9A3E0FAA3E0FB121827
:10104D007D125A4D7BD87A2A79C1783C12196EC01F
:10105D0004C005C006C0077F007E007D007C409067
:10106D00016EE0F8A3E0F9A3E0FAA3E0FB12196E1C
:10107D00A804A905AA06AB07900166E0FCA3E0FD54
:10108D00A3E0FEA3E0FF121879125A4D7B727A335A
:10109D0079DC783C12196EA804A905AA06AB079055
:1010AD000176E0FCA3E0FDA3E0FEA3E0FF121879BA
:1010BD00D003D002D001D000121879C004C005C0F1
:1010CD0006C007900172E0F8A3E0F9A3E0FAA3E0EF
:1010DD00FB900166E0FCA3E0FDA3E0FEA3E0FF12A0
:1010ED001879125A4D7B307A4C79A6783C12196ECC
:1010FD00A804A905AA06AB07D007D006D005D004D1
:10110D0012187990017612202890016EE0FCA3E070
:10111D00FDA3E0FEA3E0FF125A4D7B0B7AD2798C32
:10112D00783C12196E900176E0F8A3E0F9A3E0FA8D
:10113D00A3E0FB12187DC004C005C006C0079001D6
:10114D0072E0FCA3E0FDA3E0FEA3E0FF900166E0EA
:10115D00F8A3E0F9A3E0FAA3E0FB12187D125A4DB3
:10116D007B697AE37988783C12196EA804A905AADF
:10117D0006AB07D007D006D005D00412187D90011C
:10118D00761220287F007E007D007C4090016AE071
:10119D00F8A3E0F9A3E0FAA3E0FB12196EA804A9E5
:1011AD0005AA06AB07900166E0FCA3E0FDA3E0FEF7
:1011BD00A3E0FF121879125A4D7BF97A4E794C78CB
:1011CD003C12196EC004C005C006C007900172E044
:1011DD00FCA3E0FDA3E0FEA3E0FF125A4D7BCD7A08
:1011ED00AF79E6783B12196EA804A905AA06AB07DC
:1011FD00D007D006D005D00412187DC004C005C09C
:10120D0006C0077F007E007D007C4090016EE0F8F7
:10121D00A3E0F9A3E0FAA3E0FB12196E900172E0CE
:10122D00F8A3E0F9A3E0FAA3E0FB12187D125A4DE2
:10123D007BBC7A5779AD783B12196EA804A905AA23
:10124D0006AB07D007D006D005D00412187DC00418
:10125D00C005C006C0077F007E007D807C409001E8
:10126D006EE0F8A3E0F9A3E0FAA3E0FB12196EA873
:10127D0004A905AA06AB07900166E0FCA3E0FDA357
:10128D00E0FEA3E0FF121879125A4D7B4E7AB47925
:10129D00AB783B12196EA804A905AA06AB07D007B7
:1012AD00D006D005D00412187990017A1220287F2B
:1012BD00007E007D007C4090016EE0F8A3E0F9A374
:1012CD00E0FAA3E0FB12196EA804A905AA06AB0764
:1012DD00900166E0FCA3E0FDA3E0FEA3E0FF121881
:1012ED0079900172E0F8A3E0F9A3E0FAA3E0FB1214
:1012FD001879125A4D7BA97A6A7982783B12196E48
:10130D0090017AE0F8A3E0F9A3E0FAA3E0FB12184C
:10131D007DC004C005C006C0077F007E007D407CF7
:10132D0040900166E0F8A3E0F9A3E0FAA3E0FB1218
:10133D00196E125A4D7B9C7ADC796F783B12196EBF
:10134D00A804A905AA06AB07D007D006D005D0047E
:10135D00121879C004C005C006C0077F007E007D4D
:10136D00807C4090016EE0F8A3E0F9A3E0FAA3E0E1
:10137D00FB12196EC004C005C006C0077F007E00B9
:10138D007D007C40900166E0F8A3E0F9A3E0FAA3AC
:10139D00E0FB12196ED003D002D001D000121879E3
:1013AD00125A4D7BCA7A547941783B12196EA804B2
:1013BD00A905AA06AB07D007D006D005D004121890
:1013CD007990017A1220287F007E007D007C40906C
:1013DD00016EE0F8A3E0F9A3E0FAA3E0FB12196EA9
:1013ED00C004C005C006C0077F007E007D407C4064
:1013FD00900166E0F8A3E0F9A3E0FAA3E0FB12196F
:10140D006ED003D002D001D000121879125A4D7B44
:10141D00457A2F7923783B12196EC004C005C0069A
:10142D00C007900172E0FCA3E0FDA3E0FEA3E0FF86
:10143D0090016EE0F8A3E0F9A3E0FAA3E0FB121827
:10144D007D125A4D7B147A5C792C783B12196EA85B
:10145D0004A905AA06AB0790017AE0FCA3E0FDA361
:10146D00E0FEA3E0FF121879A804A905AA06AB07B0
:10147D00D007D006D005D00412187DC004C005C019
:10148D0006C0077F007E007D007C4090016EE0F875
:10149D00A3E0F9A3E0FAA3E0FB12196E900166E058
:1014AD00F8A3E0F9A3E0FAA3E0FB12187D90017216
:1014BD00E0F8A3E0F9A3E0FAA3E0FB121879125AC1
:1014CD004D7BA67AD57910783B12196EA804A90523
:1014DD00AA06AB07D007D006D005D004121879C0E4
:1014ED0004C005C006C0077F007E007D007C4090D3
:1014FD00016EE0F8A3E0F9A3E0FAA3E0FB12196E88
:10150D00C004C005C006C0077F007E007D007C4082
:10151D0090016AE0F8A3E0F9A3E0FAA3E0FB121949
:10152D006ED003D002D001D000121879125A4D7B23
:10153D00B37A7B79F2783A12196EA804A905AA0636
:10154D00AB07D007D006D005D00412187D90017AD4
:10155D001220287F007E007D007C4090016AE0F81B
:10156D00A3E0F9A3E0FAA3E0FB12196E900166E087
:10157D00F8A3E0F9A3E0FAA3E0FB12187DC004C0C4
:10158D0005C006C0077F007E007D007C4090016E87
:10159D00E0F8A3E0F9A3E0FAA3E0FB12196EA804AA
:1015AD00A905AA06AB07D007D006D005D00412189E
:1015BD0079125A4D7B047AAD79C0783A12196EC002
:1015CD0004C005C006C0077F007E007D007C4090F2
:1015DD000172E0F8A3E0F9A3E0FAA3E0FB12196EA3
:1015ED00C004C005C006C0077F007E007D007C40A2
:1015FD0090016EE0F8A3E0F9A3E0FAA3E0FB121965
:10160D006ED003D002D001D000121879125A4D7B42
:10161D00A37A0679D378BA12196EA804A905AA0679
:10162D00AB07D007D006D005D00412187DC004C07A
:10163D0005C006C0077F007E007D807C4090016E56
:10164D00E0F8A3E0F9A3E0FAA3E0FB12196E125A39
:10165D004D7B4B7A1F79BA783A12196EA804A905F9
:10166D00AA06AB07D007D006D005D004121879C052
:10167D0004C005C006C0077F007E007D007C409041
:10168D00016EE0F8A3E0F9A3E0FAA3E0FB12196EF6
:10169D00C004C005C006C0077F007E007D007C40F1
:1016AD00900166E0F8A3E0F9A3E0FAA3E0FB1219BC
:1016BD006ED003D002D001D000121879900172E0E3
:1016CD00F8A3E0F9A3E0FAA3E0FB12187D125A4D3E
:1016DD007BA97A3079B6783A12196EA804A905AAB1
:1016ED0006AB07D007D006D005D00412187D9001A7
:1016FD007E1220287F007E007D807C4090016EE070
:10170D00F8A3E0F9A3E0FAA3E0FB12196EA804A96F
:10171D0005AA06AB07900166E0FCA3E0FDA3E0FE81
:10172D00A3E0FF121879900172E0F8A3E0F9A3E0AD
:10173D00FAA3E0FB12187D125A4D7B3B7AAA799AD7
:10174D00783A12196EA804A905AA06AB0790017E76
:10175D00E0FCA3E0FDA3E0FEA3E0FF121879C004B6
:10176D00C005C006C0077F007E007D007C40900153
:10177D006EE0F8A3E0F9A3E0FAA3E0FB12196EC046
:10178D0004C005C006C0077F007E007D007C409030
:10179D000166E0F8A3E0F9A3E0FAA3E0FB12196EED
:1017AD00A804A905AA06AB07D007D006D005D0041A
:1017BD0012187D125A4D7B247A0B7998783A1219AA
:1017CD006EA804A905AA06AB07D007D006D005D090
:1017DD0004121879C004C005C006C0077F007E0042
:1017ED007D007C40900166E0F8A3E0F9A3E0FAA348
:1017FD00E0FB12196E900172E0F8A3E0F9A3E0FA94
:10180D00A3E0FB121879125A4D7BE07A2D7990786E
:10181D003A12196EA804A905AA06AB07D007D0067F
:10182D00D005D00412187990017E12202890017AEB
:10183D00E0FCA3E0FDA3E0FEA3E0FF900176E0F85D
:10184D00A3E0F9A3E0FAA3E0FB12187D90017EE07E
:10185D00F8A3E0F9A3E0FAA3E0FB12187D7B487A28
:08186D005179C7784512196E8C
:011875002250
:0B2B9400900120EBF0A3EAF0A3E9F0B1
:102B9F00900126E0FCA3E0FDA3E0FEA3E0FFEC1212
:102BAF001B927B007A81798878C612187D90012A52
:102BBF00E0F8A3E0F9A3E0FAA3E0FB12187D90017F
:102BCF002E1220287F0A7EEB7D157C3D90012EE092
:102BDF00F8A3E0F9A3E0FAA3E0FB12196E7B7F7A6A
:102BEF004F7940783F12187D126E119001321220EA
:102BFF00287F8C7EA67D147C3D90012EE0F8A3E00B
:102C0F00F9A3E0FAA3E0FB12196E7B367A907952A2
:102C1F00783F12187D126E119001361220287F4DC9
:102C2F007E6C7D337C3B90012EE0F8A3E0F9A3E0AE
:102C3F00FAA3E0FB12196E7B857AEA797E783F1250
:102C4F00187D126E1190013A1220287F217EB47DDB
:102C5F000A7C3D90012EE0F8A3E0F9A3E0FAA3E08F
:102C6F00FB12196E7BD37A697979783F12187D122E
:102C7F006E1190013E1220287F477E857D167C3D88
:102C8F0090012EE0F8A3E0F9A3E0FAA3E0FB1219FC
:102C9F006E7B9F7A027900783D12187D126E11902B
:102CAF0001421220287F007E007D007C4090013E73
:102CBF00E0F8A3E0F9A3E0FAA3E0FB12196E125AB1
:102CCF00637BB07A727928783F12196EC004C00501
:102CDF00C006C007900136E0FCA3E0FDA3E0FEA311
:102CEF00E0FF125A637B7D7A3F79C9784012196EE3
:102CFF00A804A905AA06AB07D007D006D005D004B3
:102D0F0012187DC004C005C006C0077F007E007D7D
:102D1F00007C4090013EE0F8A3E0F9A3E0FAA3E0C5
:102D2F00FB12196EA804A905AA06AB07900136E09D
:102D3F00FCA3E0FDA3E0FEA3E0FF121879125A6393
:102D4F007B6F7A1279A3783F12196EA804A905AA8E
:102D5F0006AB07D007D006D005D004121879C004EF
:102D6F00C005C006C00790013AE0FCA3E0FDA3E058
:102D7F00FEA3E0FF125A637BC97A76793E783E1242
:102D8F00196EA804A905AA06AB07D007D006D0056F
:102D9F00D0041218799001E2E0F8A3E0F9A3E0FA69
:102DAF00A3E0FB12196E900132E0F8A3E0F9A3E063
:102DBF00FAA3E0FB12187D900146122028900146DD
:102DCF00E0FCA3E0FDA3E0FEA3E0FFC004C005C04C
:102DDF0006C0077F007E007D007C40900142E0F836
:102DEF00A3E0F9A3E0FAA3E0FB12196E125A637B7A
:102DFF00D57A7879E9783D12196EC004C005C006FE
:102E0F00C0077F007E007D007C40900136E0F8A374
:102E1F00E0F9A3E0FAA3E0FB12196E125A637BD11B
:102E2F007A22795B783E12196ED003D002D001D08E
:102E3F0000121879C004C005C006C0077F007E00CD
:102E4F007D007C4090013EE0F8A3E0F9A3E0FAA3F7
:102E5F00E0FB12196EC004C005C006C0077F007EDC
:102E6F00007D007C40900136E0F8A3E0F9A3E0FA82
:102E7F00A3E0FB12196ED003D002D001D0001218BC
:102E8F0079125A637BFC7AA97971783D12196EA871
:102E9F0004A905AA06AB07D007D006D005D00412A7
:102EAF001879C004C005C006C0077F007E007D00F2
:102EBF007C4090013EE0F8A3E0F9A3E0FAA3E0FB29
:102ECF0012196EC004C005C006C00790013AE0FC9D
:102EDF00A3E0FDA3E0FEA3E0FF900136E0F8A3E03E
:102EEF00F9A3E0FAA3E0FB12187DD003D002D001C2
:102EFF00D000121879125A637BD57A787969783DA8
:102F0F0012196EA804A905AA06AB07D007D006D0E0
:102F1F0005D0041218799001E2E0F8A3E0F9A3E0DC
:102F2F00FAA3E0FB12196EA804A905AA06AB07D0F5
:102F3F0007D006D005D00412187D90014612202824
:102F4F007F007E007D007C4090013EE0F8A3E0F919
:102F5F00A3E0FAA3E0FB12196E125A637BE37AC760
:102F6F007928783F12196EC004C005C006C00790BB
:102F7F000136E0FCA3E0FDA3E0FEA3E0FF125A63DD
:102F8F007B9E7A5E79C7784012196EA804A905AAAC
:102F9F0006AB07D007D006D005D00412187DC004A9
:102FAF00C005C006C0077F007E007D007C409001F9
:102FBF003EE0F8A3E0F9A3E0FAA3E0FB12196EA834
:102FCF0004A905AA06AB07900136E0FCA3E0FDA318
:102FDF00E0FEA3E0FF121879125A637BE57AD079ED
:102FEF00A2783F12196EA804A905AA06AB07D0074D
:102FFF00D006D005D0041218799001E2E0F8A3E0D2
:10300F00F9A3E0FAA3E0FB12196E900142E0F8A3D6
:10301F00E0F9A3E0FAA3E0FB12187D90014A122019
:10302F00287F007E007D007C4090013EE0F8A3E009
:10303F00F9A3E0FAA3E0FB12196EA804A905AA06EA
:10304F00AB07900142E0FCA3E0FDA3E0FEA3E0FF8D
:10305F00121879125A637B067A817915783E121904
:10306F006EC004C005C006C00790014AE0FCA3E093
:10307F00FDA3E0FEA3E0FF125A637BA67A9B79A41F
:10308F00784012196ED003D002D001D000121879F7
:10309F009001E2E0F8A3E0F9A3E0FAA3E0FB121934
:1030AF006E90014E122028900146E0FCA3E0FDA394
:1030BF00E0FEA3E0FF125A63C004C005C006C007BC
:1030CF0090014EE0FCA3E0FDA3E0FEA3E0FF125A47
:1030DF004DA804A905AA06AB07D007D006D005D086
:1030EF000412196E7B327AAF79CB783E12196EC00B
:1030FF0004C005C006C00790014EE0FCA3E0FDA38D
:10310F00E0FEA3E0FF125A637BDB7ADE796A783F39
:10311F0012196EA804A905AA06AB07D007D006D0CE
:10312F0005D00412187D900123E0FBA3E0FAA3E081
:10313F00F9121FB6900123E0FBA3E0FAA3E0F91206
:10314F001F96900123E0FBA3E0FAA3E0F9122008F9
:10315F0012196EA804A905AA06AB077F007E007D91
:10316F00807C3F1218791267A29000E812202890F5
:10317F000123E0FBA3E0FAA3E0F9121F96126A2ED7
:10318F00900123E0FBA3E0FAA3E0F9121FB6900130
:10319F0046E0FCA3E0FDA3E0FEA3E0FF125A4DC002
:1031AF0004C005C006C00790014EE0FCA3E0FDA3DC
:1031BF00E0FEA3E0FF125A4DA804A905AA06AB072B
:1031CF00D007D006D005D00412196EC004C005C0B8
:1031DF0006C007900123E0FBA3E0FAA3E0F9121F5A
:1031EF0096125A4DA804A905AA06AB07D007D00618
:1031FF00D005D004121A7790015212202890014660
:10320F00E0FCA3E0FDA3E0FEA3E0FF125A63C004BD
:10321F00C005C006C00790014EE0FCA3E0FDA3E08F
:10322F00FEA3E0FF125A4DA804A905AA06AB07D0CA
:10323F0007D006D005D00412196E7BDB7ADE796ACF
:10324F00783F12196EC004C005C006C00790014E2A
:10325F00E0FCA3E0FDA3E0FEA3E0FF125A637B3284
:10326F007AAF79CB783E12196EA804A905AA06ABDE
:10327F0007D007D006D005D004121879C004C005B6
:10328F00C006C007900123E0FBA3E0FAA3E0F91208
:10329F001F96125A4DA804A905AA06AB07D007D04E
:1032AF0006D005D004121A779001561220289001EB
:1032BF0056E0FCA3E0FDA3E0FEA3E0FFC004C005C1
:1032CF00C006C007900152E0FCA3E0FDA3E0FEA3FF
:1032DF00E0FF9000E8122028D007D006D005D004D8
:1032EF00126A2E900120E0FBA3E0FAA3E0F9121F6F
:1032FF00B6900120E0FBA3E0FAA3E0F9121F967B42
:10330F00007A0079007800121B146030402E900173
:10331F0020E0FBA3E0FAA3E0F9C003C002C0011252
:10332F001F969001E6E0F8A3E0F9A3E0FAA3E0FB13
:10333F0012187DD001D002D003121FB6900120E0E9
:10334F00FBA3E0FAA3E0F9121F969001E6E0F8A3C1
:10335F00E0F9A3E0FAA3E0FB121B14502E9001201A
:10336F00E0FBA3E0FAA3E0F9C003C002C001121F03
:10337F00969001E6E0F8A3E0F9A3E0FAA3E0FB12D0
:0B338F001879D001D002D003121FB645
:01339A002210
:0B4678009001A8EBF0A3EAF0A3E9F02A
:104683009001AEE0FCA3E0FDA3E0FEA3E0FFEC128B
:104693001B927B007A81798878C612187D9001B2CB
:1046A300E0F8A3E0F9A3E0FAA3E0FB12187D7B0096
:1046B3007AAD790E7847121A779001B61220287FC7
:1046C300A67EFE7DC77C429001B6E0F8A3E0F9A385
:1046D300E0FAA3E0FB12196E7B917AEA797E783FC8
:1046E30012187D126E119001BA1220287F117E23B9
:1046F3007D5F7C379001B6E0F8A3E0F9A3E0FAA36D
:10470300E0FB12196EA804A905AA06AB077F507E29
:10471300AC7DAE7C3B121879126E11C004C005C08B
:1047230006C0079001BAE0FCA3E0FDA3E0FEA3E00E
:10473300FF125A63A804A905AA06AB07D007D0063F
:10474300D005D00412196EC004C005C006C0077F8F
:10475300187E017DC87C429001B6E0F8A3E0F9A37E
:10476300E0FAA3E0FB12196E7B327AE47946783FD4
:1047730012187D126E11A804A905AA06AB07D0076B
:10478300D006D005D00412187DC004C005C006C0F1
:10479300077F007E007D007C409001BAE0F8A3E033
:1047A300F9A3E0FAA3E0FB12196E125A637B0C7AA9
:1047B300347969783812196EA804A905AA06AB07DB
:1047C300D007D006D005D00412187D9001BE122068
:1047D300287F147E6A7D177C389001B6E0F8A3E049
:1047E300F9A3E0FAA3E0FB12196EA804A905AA062F
:1047F300AB077F6D7E6A7D857C3D121879126E1141
:104803009001C21220289001BEE0FCA3E0FDA3E0CA
:10481300FEA3E0FF125A9FC004C005C006C0079064
:1048230001C2E0FCA3E0FDA3E0FEA3E0FF125A4DAA
:10483300A804A905AA06AB07D007D006D005D00463
:1048430012196E125BAD9001A8E0FBA3E0FAA3E09E
:10485300F9121FB69001E6E0F8A3E0F9A3E0FAA38A
:10486300E0FB9001BEE0FCA3E0FDA3E0FEA3E0FFBC
:10487300121A771261FD9001E6E0F8A3E0F9A3E0D4
:10488300FAA3E0FB12196EA804A905AA06AB0790C8
:1048930001BEE0FCA3E0FDA3E0FEA3E0FF12187954
:1048A3009001C61220287F007E007DC07C3F9001CE
:1048B300EAE0F8A3E0F9A3E0FAA3E0FB12196E9093
:1048C30001C6E0F8A3E0F9A3E0FAA3E0FB121B148E
:1048D300505A7F007E007D007C3F9001EAE0F8A300
:1048E300E0F9A3E0FAA3E0FB12196E9001C6E0F829
:1048F300A3E0F9A3E0FAA3E0FB121B14402E9001FE
:10490300A8E0FBA3E0FAA3E0F9C003C002C00112D0
:104913001F969001EAE0F8A3E0F9A3E0FAA3E0FB15
:1049230012187DD001D002D003121FB69001A8E067
:10493300FBA3E0FAA3E0F9C003C002C001121F9673
:10494300C004C005C006C0079001A8E0FBA3E0FABD
:10495300A3E0F9121F969001E6E0F8A3E0F9A3E0C3
:10496300FAA3E0FB121A771261FD9001E6E0F8A3C7
:10497300E0F9A3E0FAA3E0FB12196EA804A905AAC3
:1049830006AB07D007D006D005D004121879D001A2
:10499300D002D003121FB69001BEE0FCA3E0FDA33A
:1049A300E0FEA3E0FF125A63C004C005C006C007BF
:1049B3009001C2E0FCA3E0FDA3E0FEA3E0FF125AD6
:1049C30063A804A905AA06AB07D007D006D005D073
:1049D3000412196E9001ABE0FBA3E0FAA3E0F91215
:1049E3001FB69001ABE0FBA3E0FAA3E0F9121F9618
:1049F3009001ABE0FBA3E0FAA3E0F912200812193F
:104A03006EA804A905AA06AB077F007E007D807C03
:104A13003F1218791267A29000E81220289001AB88
:104A2300E0FBA3E0FAA3E0F9121F96126A2E9001AD
:0C4A3300ABE0FBA3E0FAA3E0F9121FB611
:014A3F002254
:0B339B00900182EBF0A3EAF0A3E9F040
:1033A6007F927E0A7D867C3E900188E0F8A3E0F954
:1033B600A3E0FAA3E0FB12196E90018CE0F8A3E0FB
:1033C600F9A3E0FAA3E0FB121879900194122028E1
:1033D6007F007E007D007C00900194E0F8A3E0F978
:1033E600A3E0FAA3E0FB121B145027900194E0FC23
:1033F600A3E0FDA3E0FEA3E0FF9001E6E0F8A3E072
:10340600F9A3E0FAA3E0FB12187D9001941220289C
:1034160080489001E6E0FCA3E0FDA3E0FEA3E0FF08
:10342600900194E0F8A3E0F9A3E0FAA3E0FB121BF5
:103436001460274025900194E0FCA3E0FDA3E0FE84
:10344600A3E0FF9001E6E0F8A3E0F9A3E0FAA3E029
:10345600FB121879900194122028900194E0F8A3A9
:10346600E0F9A3E0FAA3E0FB90001EE0FCA3E0FD78
:10347600A3E0FEA3E0FF1218799000161220289010
:103486000016E0FCA3E0FDA3E0FEA3E0FF125A4D08
:10349600C004C005C006C00790001AE0FCA3E0FD0A
:1034A600A3E0FEA3E0FF125A4DA804A905AA06ABA5
:1034B60007D007D006D005D00412196EC004C00587
:1034C600C006C007900190E0FCA3E0FDA3E0FEA3C8
:1034D600E0FF125A4DA804A905AA06AB07D007D0EB
:1034E60006D005D00412196EC004C005C006C00778
:1034F60090001AE0FCA3E0FDA3E0FEA3E0FF125A51
:1035060063C004C005C006C007900190E0FCA3E0BC
:10351600FDA3E0FEA3E0FF125A63A804A905AA06CC
:10352600AB07D007D006D005D00412196EA804A99F
:1035360005AA06AB07D007D006D005D00412187D21
:10354600900198122028900198E0FCA3E0FDA3E0EA
:10355600FEA3E0FF900198E0F8A3E0F9A3E0FAA348
:10356600E0FB12196EA804A905AA06AB077F007E28
:10357600007D807C3F1218791267A290019C122070
:1035860028900198E0FCA3E0FDA3E0FEA3E0FFC0C5
:1035960004C005C006C00790019CE0FCA3E0FDA3A3
:1035A600E0FEA3E0FF9000E8122028D007D006D066
:1035B60005D004126A2E900185E0FBA3E0FAA3E091
:1035C600F9121FB6900185E0FBA3E0FAA3E0F91219
:1035D6001F96125A4DC004C005C006C0079001854B
:1035E600E0FBA3E0FAA3E0F9121F96125A63D00398
:1035F600D002D001D000121A77C004C005C006C0A0
:103606000790001AE0FCA3E0FDA3E0FEA3E0FF1292
:103616005A4DC004C005C006C00790001AE0FCA3BE
:10362600E0FDA3E0FEA3E0FF125A63D003D002D070
:1036360001D000121A77A804A905AA06AB07D0077D
:10364600D006D005D00412196EC004C005C006C04D
:1036560007900185E0FBA3E0FAA3E0F9121F96129A
:103666005A4DC004C005C006C00790001AE0FCA36E
:10367600E0FDA3E0FEA3E0FF125A4DA804A905AAA7
:1036860006AB07D007D006D005D00412196EC004C9
:10369600C005C006C007900190E0FCA3E0FDA3E0D2
:1036A600FEA3E0FF125A63D003D002D001D000126D
:1036B6001A77D003D002D001D0001218799001A455
:1036C600122028900190E0FCA3E0FDA3E0FEA3E019
:1036D600FF125A4DC004C005C006C00790001AE08C
:1036E600FCA3E0FDA3E0FEA3E0FF125A4DA804A947
:1036F60005AA06AB07D007D006D005D00412196E6E
:10370600C004C005C006C007900016E0FCA3E0FD9B
:10371600A3E0FEA3E0FF125A4DA804A905AA06AB32
:1037260007D007D006D005D00412196EC004C00514
:10373600C006C007900190E0FCA3E0FDA3E0FEA355
:10374600E0FF125A63C004C005C006C00790001A05
:10375600E0FCA3E0FDA3E0FEA3E0FF125A63A80489
:10376600A905AA06AB07D007D006D005D0041219C2
:103776006EA804A905AA06AB07D007D006D005D0C7
:103786000412187D9001A0122028900190E0FCA35D
:10379600E0FDA3E0FEA3E0FF125A4DC004C005C041
:1037A60006C007900016E0FCA3E0FDA3E0FEA3E040
:1037B600FF125A63A804A905AA06AB07D007D006CC
:1037C600D005D00412196EC004C005C006C007900B
:1037D60001A0E0FCA3E0FDA3E0FEA3E0FF9001A0B2
:1037E600E0F8A3E0F9A3E0FAA3E0FB12196EA8043F
:1037F600A905AA06AB077F007E007D807C3F1218D4
:10380600791267A2A804A905AA06AB07D007D006B5
:10381600D005D004121A779001A01220289001A09A
:10382600E0FCA3E0FDA3E0FEA3E0FFC004C005C0EA
:1038360006C0079001A4E0FCA3E0FDA3E0FEA3E020
:10384600FF9000E8122028D007D006D005D0041239
:103856006A2E900182E0FBA3E0FAA3E0F9121FB6FC
:10386600900182E0FBA3E0FAA3E0F9121F967B0029
:103876007A0079007800121B146030402E90018285
:10388600E0FBA3E0FAA3E0F9C003C002C001121FE7
:10389600969001E6E0F8A3E0F9A3E0FAA3E0FB12B4
:0B38A600187DD001D002D003121FB625
:0138B10022F4
:1066F200323B171C0205006400640001000007A37E
:106702000087038400640708038406820569000782
:1067120000020009003B003B0017001C000C006354
:1067220000C700C70002000A0E0F03840E0F038485
:106732000E0F07080E0F070800080007000E0000E2
:106742000000000000010001000000010001000043
:106752000000000000000000000000000000000037
:106762000000000000000000000000030000000321
:106772000002000300020003000300020003000203
:1067820000030000000300010003000200030002F6
:0C679200000300030002000300020003EB
:066D9900C119C11BC11A63
:106B65009000107432F0900011743BF09000127494
:106B750017F0900013741CF09000147402F090004C
:106B8500157405F012503A757900757A00D3E57AD7
:106B9500940EE57964809480503CE57A25E0FFE524
:106BA5007933FE74F82FF58274663EF583E493FC21
:106BB500740193FDE57A25E0FFE57933FE74222F14
:106BC500F58274003EF583ECF0A3EDF0057AE57AE5
:106BD5007002057980B712513E900068E4F0A3E495
:106BE500F090006AE4F0A3E4F090006CE4F0A3E414
:056BF500F012516022C6
:10422D0090003FE0F574D3E57464809482400BC335
:10423D00E574648094865002C219E5A064FFFFEF17
:10424D005407F576E5766006C29CC2988002D29C32
:10425D00E5765406FFEF60270578E578D3940A409C
:10426D000F75750AC3E57464809486500375780ADA
:10427D00E578D39414400E757564757814800675C1
:10428D007800757501AF74EF3395E0FEEF25E0FF13
:10429D00EE33FE74402FF58274673EF583E493F59B
:1042AD0072740193F573AF74EF3395E0FEEF25E073
:1042BD00FFEE33FE74162FF58274673EF583E4939B
:1042CD00F570740193F571E5746403706B900015CE
:1042DD00E0FFEF75F004121E50AFF0EF602E90006E
:1042ED0014E0FFEF3395E0FEEF25E0FFEE33FE74B3
:1042FD006A2FF58274673EF583E493FE740193FF94
:10430D00EF2571F571EE3570F570802C900014E08D
:10431D00FFEF3395E0FEEF25E0FFEE33FE74842FC3
:10432D00F58274673EF583E493FE740193FFEF25E8
:10433D0071F571EE3570F570E576B40110900028C9
:10434D00E0FEA3E0FFEF4E70040577800375770064
:10435D00E577C394144008757700A219B39219D369
:10436D00E57664809481500302461CC3E574648035
:10437D009486400302444212508FE57664047055D2
:10438D00AF74EF3395E0FE74102FF58274003EF597
:10439D0083E02575F0AF74EF3395E0FE74102FF5C3
:1043AD008274003EF583E0FFEF3395E0FED3EF9589
:1043BD0071E5706480F8EE6480984016AF73AE744A
:1043CD00EEFD3395E0FC74102DF58274003CF58301
:1043DD00EFF012503AE5766402705AAF74EF3395F0
:1043ED00E0FE74102FF58274003EF583E0FFC3EFFD
:1043FD009575FFEFF0AF74EF3395E0FE74102FF568
:10440D008274003EF583E0FFEF3395E0FEC3EF9538
:10441D0073E5726480F8EE6480985016AF71AE74D7
:10442D00EEFD3395E0FC74102DF58274003CF583A0
:10443D00EFF012503AC3E574648094865003024540
:10444D005E74FA2574F574E57664047072AF75EFD9
:10445D00FD7C00AF74EF3395E0FEEF25E0FFEE330A
:10446D00FE74222FF58274003EF583EC8DF0121F41
:10447D0012AF74EF3395E0FEEF25E0FFEE33FE74DF
:10448D00222FF58274003EF583E0FEA3E0FFD3EF0B
:10449D009571E5706480F8EE648098401FAF74EFFD
:1044AD003395E0FEEF25E0FFEE33FE74222FF5820B
:1044BD0074003EF583E572F0A3E573F012513EE50D
:1044CD007664026003024558AF74EF3395E0FEEF5A
:1044DD0025E0FFEE33FE74222FF58274003EF58346
:1044ED00C083C082E0FEA3E0FFAD757C00C3EF9DED
:1044FD00FFEE9CFED082D083EEF0A3EFF0AF74EF11
:10450D003395E0FEEF25E0FFEE33FE74222FF582AA
:10451D0074003EF583E0FEA3E0FFC3EF9573E572F3
:10452D006480F8EE648098501FAF74EF3395E0FE11
:10453D00EF25E0FFEE33FE74222FF58274003EF579
:10454D0083E570F0A3E571F012513E74062574F504
:10455D0074900028E0FEA3E0FFEF4E705CE576B4AA
:10456D000526301B230574AF74D3EF6480949340FC
:10457D0003757400C21BAF74EF3395E0FE90003EDF
:10458D00EEF0A3EFF012513EE576640360030246B0
:10459D001C301B7B1574AF74C3EF64809480500383
:1045AD00757413C21BAF74EF3395E0FE90003EEEB1
:1045BD00F0A3EFF012513E8056E576B40526301B80
:1045CD00230574AF74D3EF64809492400375740027
:1045DD00C21BAF74EF3395E0FE90003EEEF0A3EFFB
:1045ED00F012513EE576B40326301B231574AF74DB
:1045FD00C3EF648094805003757412C21BAF74EFC7
:10460D003395E0FE90003EEEF0A3EFF012513EE543
:10461D0076B40102D21BE5765406FFEF60109000D0
:10462D003EE0FEA3E0FFEF64094E7002C20F900260
:10463D0005E0FEA3E0FF900028E0FCA3E0FDED6F98
:10464D007002EC6E6002C20F900028E0FEA3E0FF46
:10465D00900205EEF0A3EFF030A302D21A20A30AC8
:0A466D00301A07C21AA20FB3920F11
:014677002220
:10503A001251A974A01251C174021251C1900010E8
:10504A007C03E01251821251C1A3DCF6E0125182B4
:10505A00F5F0A3A3E0030354C045F01251C1900038
:10506A0014E01251821251C1C2B412519C1251A9B8
:10507A0074A01251C174F01251C1A3E01251C1C2FD
:10508A00B412519C221251A974A01251C174021275
:10509A0051C11251A974A0041251C19000101251A9
:1050AA00E612518AF0A31251F91251E612518AF00E
:1050BA00A31251F91251E612518AF0A31251F912B0
:1050CA0051E6FB543F12518AF0A31251F91251E6EC
:1050DA00FA541F12518AF0EB23235403FD1251F3A1
:1050EA00C2B412519C1251A974A01251C174F01287
:1050FA0051C11251A974A0041251C11251E6FB54B4
:10510A0003C39D2405838007030201000302012BC8
:10511A00A3F0F5F01251F3C2B412519C1251A974C2
:10512A00A01251C174F01251C1E5F01251C1C2B4BA
:10513A0012519C227AA07B807C1E90002212523946
:10514A00227AA07B80125201ED900022F07AA0A36D
:10515A007C1D12526E227AA07BD07C1090006812BD
:10516A005239227AA07BD0125201ED900068F07A6F
:01517A00A094
:10517B00A37C0F12526E2275F00A84C425F022C054
:10518B00E0C4540F75F00AA4F5F0D0E0540F25F0ED
:10519B002200D2B5000000D2B40000000022125150
:1051AB009CC2B4000000C2B500000022D2B50000C2
:1051BB0000C2B50000227E083392B41251B7DEF85C
:1051CB0033D2B40000A2B450040000A2B41251B701
:1051DB00400122C2B4000012519C227E08A2B433BB
:1051EB00001251B7DEF7C322D2B41251B722C2B4A8
:1051FB001251B7D2B4221251A9EA1251C1EB12517A
:10520B00C11251A9EA041251C11251E6FD1251F318
:10521B00C2B412519C221251A9EA1251C1EB125184
:10522B00C1E61251C108DCF9C2B412519C221251D1
:10523B00A9EA1251C1EB1251C1E01251C1A3DCF921
:10524B00C2B412519C221251A9EA041251C180031B
:10525B001251F91251E6F608DCF61251F3C2B412F0
:10526B00519C221251A9EA041251C180031251F927
:0C527B001251E6F0A3DCF61251F3C2B4AD
:0452870012519C2202
:104D4000202020202531642E253032642025303269
:104D500062753A25303262753A253032627520200C
:104D600020200020202020253032642E2531642090
:104D700025303262753A25303262753A253032621A
:104D8000752020202000253033642E25316420201A
:104D9000253032642E25316420415A2F454C312074
:104DA000202000253033642E253164202025303228
:104DB000642E25316420415A2F454C32202020009A
:104DC000253033642E2531642020253032642E2591
:104DD00031642052412F44454320202000253033A8
:104DE000642E2531645720253032642E2531644EDF
:104DF000204C4F2F4C41202020002530326275205E
:104E000020202530326275202025303262753A2507
:104E1000303262753A25303262752020202000251C
:104E200030352E31662020253032642E2531642025
:104E300020202020202025303264202000202B2517
:104E40003031642E2530316420202B253031642E02
:104E50002530316420434F52202053545020002DE0
:104E60002D2D2D2D2D2D2D2D2D2D202020202020C0
:104E70005354502000253033642E253164202025E2
:104E80003032642E25316420414E54202025316477
:104E90002E2531642000202020204F204520352061
:104EA0004A2046204C2020202020002020202020A6
:104EB000202020454D45202020202020202020009B
:104EC00020416E74656E6E6120436F6E74726F6CFC
:104ED0006C65722000202020202020207620372E94
:104EE000332020202020202020002020204A414E56
:104EF0004645424D41524150524D41594A554E4A04
:104F0000554C4155475345504F43544E4F564445D9
:104F100043004D4F4F4E202053554E2020204341FB
:104F20005353494F4359474E55535341474954549E
:104F30005441555255534C454F2020204151554125
:104F4000522E52412F444543415A2F454C32415A2B
:104F50002F454C3100326D3A37303A32333A3133E3
:104F60003A39636D36636D31304732344700205330
:104F7000534920313062697428373230292020208B
:104F80002020205353493131626974283138303040
:104F9000292020202020205353493132626974286F
:104FA00033363030292020202020205353495F679A
:104FB0007261792834303936292020202020204180
:104FC000322D532D5320313220626974202020204D
:104FD00020204D414232355F3130626974313032C8
:104FE0003420202020204D414232355F313162692A
:104FF000743230343820202020204D414232355F39
:1050000031326269743430393620202020204D41FD
:105010004232385F313262697434303936202020B0
:105020002020000F0C09010306171D664C0309031D
:0A50300009030903095601010204F7
:10002E00E57664016003125D75201403020663C257
:10003E001430190C900028E0FEA3E0FFEF4E601183
:10004E0090003EE0FEA3E0FFEF64134E600302015A
:10005E00FB90003CE0FEA3E0FFC3EF9404EE64804F
:10006E0094804003020108AF1CAE1B126ED2EF2427
:10007E0005FFEE3400FE7C007D0A121EDC9000E0CF
:10008E00EEF0A3EFF07B017A007980C003C002C0CE
:10009E00017BFF7A4D79409000F3EBF0A3EAF0A3D9
:1000AE00E9F09000E0E0FEA3E0FF7C007D64121E0C
:1000BE00DC9000F6EEF0A3EFF09000E0E0FEA3E09F
:1000CE00FF7C007D64121EDC9000F8ECF0A3EDF0D6
:1000DE00900012E0FF9000FAEFF0900011E0FF9018
:1000EE0000FBEFF0900010E0FF9000FCEFF0D0016D
:1000FE00D002D003123E0F020198AF1CAE1B126E3F
:10010E00D2EF2405FFEE3400FE7C007D0A121EDCC9
:10011E009000E0EEF0A3EFF07B017A007980C0034F
:10012E00C002C0017BFF7A4D79639000F3EBF0A320
:10013E00EAF0A3E9F09000E0E0FEA3E0FF7C007D92
:10014E000A121EDC9000F6EEF0A3EFF09000E0E055
:10015E00FEA3E0FF7C007D0A121EDC9000F8ECF09E
:10016E00A3EDF0900012E0FF9000FAEFF090001176
:10017E00E0FF9000FBEFF0900010E0FF9000FCEF2E
:10018E00F0D001D002D003123E0F751500D3E51545
:10019E00648094825042AF1590003DE0FE75F003EE
:1001AE00EEA4F58285F083E5822FF582E43583F5A2
:1001BE0083E5822455F582E583344FF583E493FF7E
:1001CE00AE15EEFD3395E0FC74802DF58274003C87
:1001DE00F583EFF0051580B5C3E51B648094804070
:1001EE00030205F3900083742DF00205F390003E98
:1001FE00E0FEA3E0FFEF640A4E601190003EE0FEC9
:10020E00A3E0FFEF640B4E600302029F7B017A00B6
:10021E007980C003C002C0017BFF7A4D79869000C1
:10022E00F3EBF0A3EAF0A3E9F090002AE0FEA3E0DE
:10023E00FF7C007D0A121EDC9000F6EEF0A3EFF0BC
:10024E0090002AE0FEA3E0FF7C007D0A121EDC90E7
:10025E0000F8ECF0A3EDF090002CE0FEA3E0FF7CA4
:10026E00007D0A121EDC9000FAEEF0A3EFF0900073
:10027E002CE0FEA3E0FF7C007D0A121EDC9000FC49
:10028E00ECF0A3EDF0D001D002D003123E0F020528
:10029E00F390003EE0FEA3E0FFEF640C4E60119081
:1002AE00003EE0FEA3E0FFEF640D4E600302034349
:1002BE007B017A007980C003C002C0017BFF7A4DBA
:1002CE0079A39000F3EBF0A3EAF0A3E9F090002EEF
:1002DE00E0FEA3E0FF7C007D0A121EDC9000F6EE2D
:1002EE00F0A3EFF090002EE0FEA3E0FF7C007D0A6D
:1002FE00121EDC9000F8ECF0A3EDF0900030E0FE62
:10030E00A3E0FF7C007D0A121EDC9000FAEEF0A343
:10031E00EFF0900030E0FEA3E0FF7C007D0A121E9D
:10032E00DC9000FCECF0A3EDF0D001D002D0031273
:10033E003E0F0205F390003EE0FEA3E0FFEF640ED9
:10034E004E601190003EE0FEA3E0FFEF640F4E60A2
:10035E0003020426900034E0FEA3E0FFEF247CFFAE
:10036E00EE34FCFE90007CEEF0A3EFF090007CE00B
:10037E00FEA3E0FF126ED27C007D0A121EDCC006C8
:10038E00C00790007CE0FEA3E0FF126ED27C007DE1
:10039E000A121EDC9000FCECF0A3EDF0D007D006A4
:1003AE009000FAEEF0A3EFF07B017A007980C003A3
:1003BE00C002C0017BFF7A4D79C09000F3EBF0A331
:1003CE00EAF0A3E9F0900032E0FEA3E0FF7C007DAE
:1003DE000A121EDC9000F6EEF0A3EFF0900032E071
:1003EE00FEA3E0FF7C007D0A121EDC9000F8ECF00C
:1003FE00A3EDF0D001D002D003123E0F90007CE0AE
:10040E00FEA3E0FFC3EE6480948040030205F390E8
:10041E000086742DF00205F390003EE0FEA3E0FF8F
:10042E00EF64104E601190003EE0FEA3E0FFEF641B
:10043E00114E600302054D900036E0FEA3E0FFEF83
:10044E0024F8FFEE34F8FE90007EEEF0A3EFF0906D
:10045E000038E0FEA3E0FFEF247CFFEE34FCFE90BC
:10046E00007CEEF0A3EFF090007EE0FEA3E0FF1222
:10047E006ED27C007D0A121EDCC006C00790007E84
:10048E00E0FEA3E0FF126ED27C007D0A121EDCC0DD
:10049E0004C00590007CE0FEA3E0FF126ED27C004B
:1004AE007D0A121EDCC006C00790007CE0FEA3E0B1
:1004BE00FF126ED27C007D0A121EDC9000FCECF066
:1004CE00A3EDF0D007D0069000FAEEF0A3EFF0D037
:1004DE0005D0049000F8ECF0A3EDF0D007D0069014
:1004EE0000F6EEF0A3EFF07B017A007980C003C036
:1004FE0002C0017BFF7A4D79DD9000F3EBF0A3EAA9
:10050E00F0A3E9F0D001D002D003123E0F90007E8E
:10051E00E0FEA3E0FFC3EE64809480500690008559
:10052E007445F090007CE0FEA3E0FFC3EE6480947F
:10053E008040030205F390008B7453F00205F37BA9
:10054E00017A007980C003C002C0017BFF7A4D7929
:10055E00FA9000F3EBF0A3EAF0A3E9F0900013E0B9
:10056E00FF9000F6EFF0900015E0FF9000F7EFF02F
:10057E00900012E0FF9000F8EFF0900011E0FF9075
:10058E0000F9EFF0900010E0FF9000FAEFF0D001CC
:10059E00D002D003123E0F751500D3E5156480947A
:1005AE00825042AF15900014E0FE75F003EEA4F5F4
:1005BE008285F083E5822FF582E43583F583E5822B
:1005CE0024EAF582E583344EF583E493FFAE15EE0F
:1005DE00FD3395E0FC74822DF58274003CF583EFBB
:1005EE00F0051580B5900028E0FEA3E0FFC3EF9460
:1005FE0002EE64809480503290003EE0FEA3E0FF55
:10060E00C3EF940AEE64809480401390003EE0FEA7
:10061E00A3E0FFD3EF9411EE64809480400C900021
:10062E00927444F09000937445F07F00125D8775CC
:10063E001500D3E51564809493501AAF15EF3395DA
:10064E00E0FE74802FF58274003EF583E0FF125DAC
:10065E004E051580DD201503020879C21590003E67
:10066E00E0FEA3E0FFC3EF940AEE64809480401591
:10067E0090003EE0FEA3E0FFD3EF9411EE64809471
:10068E00805002C2199001E2E0F8A3E0F9A3E0FA6B
:10069E00A3E0FB900004E0FCA3E0FDA3E0FEA3E0DA
:1006AE00FF121A77126F397B007A00792078411287
:1006BE00196E7B007A007900783F12187D121BD0DC
:1006CE0090007CEEF0A3EFF09001E2E0F8A3E0F9E9
:1006DE00A3E0FAA3E0FB900078E0FCA3E0FDA3E02A
:1006EE00FEA3E0FF121A77126F397B007A007900B1
:1006FE00783F12187D121BD09000E2EEF0A3EFF0BF
:10070E007B017A007998C003C002C0017BFF7A4E4C
:10071E00791F9000F3EBF0A3EAF0A3E9F09001E269
:10072E00E0F8A3E0F9A3E0FAA3E0FB90000CE0FCF4
:10073E00A3E0FDA3E0FEA3E0FF121A779000F612ED
:10074E00202890007CE0FEA3E0FF7C007D0A121EB4
:10075E00DC9000FAEEF0A3EFF090007CE0FEA3E058
:10076E00FF7C007D0A121EDC9000FCECF0A3EDF085
:10077E009000E2E0FEA3E0FF9000FEEEF0A3EFF0AB
:10078E00D001D002D003123E0F7F007E007D007C90
:10079E0000900004E0F8A3E0F9A3E0FAA3E0FB1256
:1007AE001B14500690009E742DF0751500D3E515A0
:1007BE00648094855042AF15900029E0FE75F006D6
:1007CE00EEA4F58285F083E5822FF582E43583F57C
:1007DE0083E5822412F582E583344FF583E493FF9B
:1007EE00AE15EEFD3395E0FC74A42DF58274003C3D
:1007FE00F583EFF0051580B5900028E0FEA3E0FF2D
:10080E00C3EF9402EE64809480400E9000AA742090
:10081E00F09000AB7420F080217F007E007D007C84
:10082E0000900078E0F8A3E0F9A3E0FAA3E0FB1251
:10083E001B1450069000A9742DF0E5766401602B10
:10084E007F40125D87751500D3E515648094935033
:10085E001AAF15EF3395E0FE74982FF58274003EB3
:10086E00F583E0FF125D4E051580DD2016030209AB
:10087E00CAC216900022E0FEA3E0FFEF249CFFEE1A
:10088E0034FFFE126ED290007EEEF0A3EFF09000D9
:10089E0024E0FEA3E0FFEF249CFFEE34FFFE126E79
:1008AE00D290007CEEF0A3EFF03010030209417BF2
:1008BE00017A0079B0C003C002C0017BFF7A4E7985
:1008CE003D9000F3EBF0A3EAF0A3E9F090007EE098
:1008DE00FEA3E0FF7C007D0A121EDC9000F6EEF017
:1008EE00A3EFF090007EE0FEA3E0FF7C007D0A12F5
:1008FE001EDC9000F8ECF0A3EDF090007CE0FEA37F
:10090E00E0FF7C007D0A121EDC9000FAEEF0A3EFF1
:10091E00F090007CE0FEA3E0FF7C007D0A121EDC5E
:10092E009000FCECF0A3EDF0D001D002D003123E0B
:10093E000F80267B017A0079B0C003C002C0017B14
:10094E00FF7A4E795F9000F3EBF0A3EAF0A3E9F0A3
:10095E00D001D002D003123E0F900022E0FEA3E0A1
:10096E00FFC3EF9464EE6480948050069000B174DF
:10097E002DF0900024E0FEA3E0FFC3EF9464EE643C
:10098E0080948050069000B7742DF0E57664016077
:10099E002B7F14125D87751500D3E5156480949333
:1009AE00501AAF15EF3395E0FE74B02FF582740038
:1009BE003EF583E0FF125D4E051580DD2017030224
:1009CE000BE3C217900027E0FFEF90503793FFEF35
:1009DE003395E0FEAC66AD67121ECA8E4A8F4B9001
:1009EE0001F9E0FEA3E0FF126ED27C007D0A121E1A
:1009FE00DCC006C0079001F9E0FEA3E0FF126ED244
:100A0E007C007D0A121EDC9000FCECF0A3EDF0D011
:100A1E0007D0069000FAEEF0A3EFF07B017A007992
:100A2E00C8C003C002C0017BFF7A4E79759000F3F7
:100A3E00EBF0A3EAF0A3E9F09001FBE0FEA3E0FFE8
:100A4E007C007D0A121EDC9000F6EEF0A3EFF09013
:100A5E0001FBE0FEA3E0FF7C007D0A121EDC90008D
:100A6E00F8ECF0A3EDF0AE4AAF4B7C007D0A121EFF
:100A7E00DC9000FEEEF0A3EFF0AE4AAF4B7C007DB3
:100A8E000A121EDC900100ECF0A3EDF0D001D002B2
:100A9E00D003123E0F9001F9E0FEA3E0FFC3EE6417
:100AAE0080948050069000CE742DF0A21CB3921C40
:100ABE00E508540CFFEFB40808201C059000D8E49C
:100ACE00F0E508540CFFEFB40409201C069000D882
:100ADE007401F0E508540CFFEFB40C09300F0690CA
:100AEE0000D8742AF0E5085403FFEFB40209301C55
:100AFE00069000D77402F0E5085403FFEFB4010925
:100B0E00301C069000D77403F0E5085403FFEFB4D1
:100B1E000309300F069000D7742AF090003EE0FED5
:100B2E00A3E0FFEF64124E6003020BB8751500D3FD
:100B3E00E515648094935042AF1590003BE0FE752E
:100B4E00F014EEA4F58285F083E5822FF582E4356C
:100B5E0083F583E582246EF582E583344FF583E4D5
:100B6E0093FFAE15EEFD3395E0FC74C82DF582743F
:100B7E00003CF583EFF0051580B5AE4AAF4B7C0017
:100B8E007D0A121EDCEF2430FF9000D9EFF09000AA
:100B9E00DA742EF0AE4AAF4B7C007D0A121EDCAF2B
:100BAE0005EF2430FF9000DBEFF07F54125D877568
:100BBE001500D3E51564809493501AAF15EF339555
:100BCE00E0FE74C82FF58274003EF583E0FF125DDF
:100BDE004E051580DDE576B4011490003FE0FFEF81
:100BEE0090502393FF125D87125D6C125D7E30185C
:100BFE0003020D467B017A007980C003C002C0015A
:100C0E007BFF7A4E79969000F3EBF0A3EAF0A3E91E
:100C1E00F0D001D002D003123E0F7B017A007998FA
:100C2E00C003C002C0017BFF7A4E79AB9000F3EB9C
:100C3E00F0A3EAF0A3E9F0D001D002D003123E0FE8
:100C4E007B017A0079B0C003C002C0017BFF7A4EEF
:100C5E0079C09000F3EBF0A3EAF0A3E9F0D001D055
:100C6E0002D003123E0F7B017A0079C8C003C00286
:100C7E00C0017BFF7A4E79D59000F3EBF0A3EAF03A
:100C8E00A3E9F0D001D002D003123E0F7F00125D17
:100C9E0087751500D3E51564809493501AAF15EF40
:100CAE003395E0FE74802FF58274003EF583E0FFED
:100CBE00125D4E051580DD7F40125D87751500D3E0
:100CCE00E51564809493501AAF15EF3395E0FE74DA
:100CDE00982FF58274003EF583E0FF125D4E0515E8
:100CEE0080DD7F14125D87751500D3E51564809441
:100CFE0093501AAF15EF3395E0FE74B02FF5827452
:100D0E00003EF583E0FF125D4E051580DD7F541227
:100D1E005D87751500D3E51564809493501AAF1551
:100D2E00EF3395E0FE74C82FF58274003EF583E034
:090D3E00FF125D4E051580DD2257
:106D9F00015100014F00015000014900C10FC10C0A
:0A6DAF00C10BC10EC110C10DC111CE
:106EE400752400D3E524648094A75004052480F31A
:016EF400227B
:106EF500752500D3E525648094935004052580F31A
:016F05002269
:106F0600752600D3E5266480949E5004052680F3FA
:016F16002258
:106F1700752700D3E5276480949E5004052780F3E6
:016F27002247
:106F2800752800D3E5286480949E5004052880F3D2
:016F38002236
:10610400C290126EE4752E1F752D00E52DD39407F1
:106114005011E52EC313F52EA2D79290126EE4050A
:106124002D80E8D290126EE4D292752903752AE884
:10613400752E00309110E52A152A7002152914FFD6
:10614400AE29EF4E70ED126EF5752D00E52DD3944A
:10615400075013126EE4E52EC313F52E309103435A
:106164002E80052D80E6126EE4AF2E7E00EF752C96
:1061740000F52B752903752AE8752E00309110E57A
:106184002A152A7002152914FFAE29EF4E70ED125C
:106194006EF5752D00E52DD394075013126EE4E5CA
:1061A4002EC313F52E309103432E80052D80E61265
:1061B4006EE4AF2E7E00EF252CF52CEE352BF52B5F
:1061C400C3E52B648094805006752B00752C00D396
:1061D400E52C940FE52B6480948E4006752B0E7588
:1061E4002C0FC29220B20DC3740F952CF52C740E93
:0861F400952BF52BAE2BAF2C0F
:0161FC002280
:1063DB00C294126EE475341F753300E533D3940702
:1063EB005011E534C313F534A2D79294126EE40521
:1063FB003380E8D294126EE4D296752F037530E891
:10640B00753400309510E53015307002152F14FFE0
:10641B00AE2FEF4E70ED126EF5753300E533D3945E
:10642B00075013126EE4E534C313F5343095034370
:10643B003480053380E6126EE4AF347E00EF7532A4
:10644B0000F531752F037530E8753400309510E584
:10645B003015307002152F14FFAE2FEF4E70ED126A
:10646B006EF5753300E533D394075013126EE4E5E4
:10647B0034C313F534309503433480053380E6126F
:10648B006EE4AF347E00EF2532F532EE3531F53167
:10649B00C3E531648094805006753100753200D3AA
:1064AB00E532940FE5316480948E400675310E759C
:0864BB00320FC296AE31AF3280
:0164C30022B6
:10000E001261048E4D8F4E1263DB8E478F487566DC
:05001E000075670122DE
:1068EF00D290D294D291D295756C00756D00756867
:1068FF0000756900753500D3E5356480948950497A
:10690F00126F06C290C294126F06C3E5356480946D
:10691F00895004D290D294E56D256DF56DE56C35F7
:10692F006CF56CE5692569F569E5683568F56820EA
:10693F009108056DE56D7002056C2095080569E5F8
:10694F006970020568053580AEC290C29475660005
:10695F00756705AE6CAF6D7C007D05121ECA8E4D3E
:10696F008F4E20B20DC3740B954EF54E740E954D90
:10697F00F54DAE68AF697C007D05121ECA8E478F3C
:01698F0048BF
:0169900022E4
:106ACB00D290D294D291D295756C00756D00756889
:106ADB0000756900753600D3E5366480948A504999
:106AEB00126F06C290C294126F06C3E5366480948F
:106AFB008A5004D290D294E56D256DF56DE56C3519
:106B0B006CF56CE5692569F569E5683568F568200C
:106B1B009108056DE56D7002056C2095080569E51A
:106B2B006970020568053680AEC290C29475660026
:106B3B00756702E56D25E0F54EE56C33F54D20B23A
:106B4B000DC3740E954EF54E740E954DF54DE569CE
:096B5B0025E0F548E56833F54733
:016B6400220E
:106C8B00D290D294D291D295756C00756D007568C7
:106C9B0000756900753700D3E5376480948B5049D4
:106CAB00126F06C290C294126F06C3E537648094CC
:106CBB008B5004D290D294E56D256DF56DE56C3556
:106CCB006CF56CE5692569F569E5683568F568204B
:106CDB009108056DE56D7002056C2095080569E559
:106CEB006970020568053780AEC290C29475660064
:106CFB00756701856C4D856D4E20B20DC3740F9574
:0F6D0B004EF54E740E954DF54D856847856948D8
:016D1A002256
:105DCC00D292D291756C00756D00126F17753800F8
:105DDC00D3E5386480948F5025D290126F17C290FF
:105DEC00126F17E56D256DF56DE56C356CF56C2056
:105DFC009108056DE56D7002056C053880D2C29076
:105E0C00C292E56DAE6C7806CEC313CE13D8F9F5FD
:105E1C006D8E6CAC6CAD6DE4121B977B007A0079C7
:105E2C0034784412196E7B007A0079807844121A07
:105E3C0077121BD07C007D05121ECA8E4D8F4E2012
:105E4C00B20DC3740B954EF54E740E954DF54D1267
:105E5C006F17756600756705D296D29575680075D3
:105E6C006900126F17753800D3E5386480948F5031
:105E7C0025D294126F17C294126F17E5692569F534
:105E8C0069E5683568F5682095080569E56970026B
:105E9C000568053880D2C294C296E569AE6878066A
:105EAC00CEC313CE13D8F9F5698E68AC68AD69E42E
:105EBC00121B977B007A007934784412196E7B00A0
:105ECC007A0079807844121A77121BD07C007D05F9
:075EDC00121ECA8E478F4819
:015EE300229C
:105EE400D292D291756C00756D00126F17753900DE
:105EF400D3E5396480948F5025D290126F17C290E5
:105F0400126F17E56D256DF56DE56C356CF56C203C
:105F14009108056DE56D7002056C053980D2C2905B
:105F2400C292E56DAE6C7805CEC313CE13D8F9F5E5
:105F34006D8E6CAC6CAD6DE4121B977B007A0079AE
:105F4400E1784412196E7B007A0079007845121AC0
:105F540077121BD0EF25E0F54EEE33F54D20B20D50
:105F6400C3740E954EF54E740E954DF54D126F1784
:105F7400756600756702D296D295756800756900DA
:105F8400126F17753900D3E5396480948F5025D288
:105F940094126F17C294126F17E5692569F569E5C4
:105FA400683568F5682095080569E5697002056833
:105FB400053980D2C294C296E569AE687805CEC32D
:105FC40013CE13D8F9F5698E68AC68AD69E4121B79
:105FD400977B007A0079E1784412196E7B007A008D
:105FE40079007845121A77121BD0EF25E0F548EEB8
:035FF40033F5473B
:015FF7002287
:105FF800D292D291756C00756D00126F17753A00C8
:10600800D3E53A6480948F5025D290126F17C290CE
:10601800126F17E56D256DF56DE56C356CF56C2027
:106028009108056DE56D7002056C053A80D2C29045
:10603800C292E56CC4F854F0C868F56CE56DC454B8
:106048000F48F56DAC6CAD6DE4121B977B007A00C0
:106058007961784512196E7B007A0079807845124B
:106068001A77121BD08E4D8F4E20B20DC3740F9528
:106078004EF54E740E954DF54D126F1775660075F9
:106088006701D296D295756800756900126F177509
:106098003A00D3E53A6480948F5025D294126F1752
:1060A800C294126F17E5692569F569E5683568F5E1
:1060B800682095080569E56970020568053A80D287
:1060C800C294C296E568C4F854F0C868F568E569F2
:1060D800C4540F48F569AC68AD69E4121B977B009E
:1060E8007A007961784512196E7B007A0079807898
:0B60F80045121A77121BD08E478F480C
:016103002279
:10586100D292D291756C00756D00126F28753B0054
:10587100D3E53B6480948F5025D290126F28C2905B
:10588100126F28E56D256DF56DE56C356CF56C20B5
:105891009108056DE56D7002056C053B80D2C290E3
:1058A100C292E56CC4F854F0C868F56CE56DC45457
:1058B1000F48F56DD3E56D9559E56C955840188500
:1058C1006C62856D63856C58856D59E56D24FFF5B6
:1058D10057E56C34FFF556C3E56D9557E56C955664
:1058E100501EE56D2401F563E56C3400F562856CAD
:1058F10056856D57E56D2401F559E56C3400F55871
:10590100AC62AD63EC121B977B007A00796178453C
:1059110012196E7B007A0079807845121A77121B72
:10592100D08E4D8F4E20B20DC3740F954EF54E742F
:105931000E954DF54D126F17756600756701D2967C
:10594100D295756800756900126F28753B00D3E523
:105951003B6480948F5025D294126F28C294126FA9
:1059610028E5692569F569E5683568F568209508D0
:105971000569E56970020568053B80D2C294C2964B
:10598100E568C4F854F0C868F568E569C4540F487F
:10599100F569D3E5699555E5689554401885685EC4
:1059A10085695F856854856955E56924FFF553E587
:1059B1006834FFF552C3E5699553E5689552501E69
:1059C100E5692401F55FE5683400F55E8568528577
:1059D1006953E5692401F555E5683400F554AC5E79
:1059E100AD5FEC121B977B007A0079617845121943
:1059F1006E7B007A0079807845121A77121BD08E5F
:035A0100478F4884
:015A0400227F
:1062ED00D290D294D291D295756C00756D0075686F
:1062FD0000756900753C00D3E53C6480948B505368
:10630D00C290C294753D00D3E53D648094825004E3
:10631D00053D80F3C3E53C6480948B5004D290D24C
:10632D0094E56D256DF56DE56C356CF56CE56925C0
:10633D0069F569E5683568F568209108056DE56DC5
:10634D007002056C2095080569E569700205680500
:10635D003C80A4C290C294756600756701AF6DAEA6
:10636D006C126EBA8E6C8F6DAF69AE68126EBA8E8E
:10637D00688F69AC6CAD6DE4121B977B007A007968
:10638D0061784512196E7B007A0079807845121A72
:10639D0077121BD08E4D8F4E20B20DC3740F954EBC
:1063AD00F54E740E954DF54DAC68AD69E4121B9725
:1063BD007B007A007961784512196E7B007A00793D
:0D63CD00807845121A77121BD08E478F483A
:0163DA0022A0
:1038B200E54C64326003300D61C3E56F954EF561EE
:1038C200E56E954DF560C374089548FF74079547FA
:1038D200FE126ED2C374849FFF74039EFEC3E56B17
:1038E2009FF55BE56A9EF55AC3E5489408E547648F
:1038F200809487400BC3E4955BF55BE4955AF55AD7
:10390200C210C20E900068E560F0A3E561F090007D
:103912006AE55AF0A3E55BF0C20D20101B20B30349
:10392200300E03301112D210D20E90006CE4F0A3CC
:103932007401F0125160C21130101D20B303300E19
:1039420003301114C210D20E12514B90006CE4F0ED
:10395200A3E4F0125160C21120B304054C80057536
:103962004C00C20E301074E561254EF54EE560350F
:103972004DF54DD3E54E940FE54D6480948E400C89
:1039820074F0254EF54E74F1354DF54DC3E54D6499
:10399200809480500C7410254EF54E740E354DF502
:1039A2004DE55B2548F548E55A3547F547D3E548E7
:1039B200940FE5476480948E400C74F02548F548D6
:1039C20074F13547F547C3E54764809480500C7421
:1039D200102548F548740E3547F547C374089548D5
:1039E200FF74079547FE126ED2C374849FF5487424
:1039F200039EF5479001FBE54DF0A3E54EF09001E3
:103A0200F9E547F0A3E548F0E56F24F8F55DE56ECA
:103A120034F8F55CE54E24F8F565E54D34F8F564C7
:103A2200C3E55C64809480500C7410255DF55D7470
:103A32000E355CF55CC3E56464809480500C7410B0
:103A42002565F565740E3564F56430105A900038BA
:103A5200E0FEA3E0FFC3EF9484EE64809483400F02
:103A6200C3E56F954EF53FE56E954DF53E800DC36E
:103A7200E55D9565F53FE55C9564F53ED3E56B94B0
:103A820000E56A648094804010C3E56B9548F54177
:103A9200E56A9547F540023B51C3E49548F541E498
:103AA2009547F540023B51900038E0FEA3E0FFC38A
:103AB200EF9484EE648094834025900022E0FEA37C
:103AC200E0FFE56F2FFFE56E3EFEEF249CFFEE3434
:103AD200FFFEC3EF954EF53FEE954DF53E802390E8
:103AE2000022E0FEA3E0FFE55D2FFFE55C3EFEEF76
:103AF200249CFFEE34FFFEC3EF9565F53FEE95641F
:103B0200F53ED3E56B9400E56A648094804025908D
:103B12000024E0FEA3E0FFE56B2FFFE56A3EFEEF27
:103B2200249CFFEE34FFFEC3EF9548F541EE954726
:103B3200F540801B900024E0FEA3E0FFEF249CFFF1
:103B4200EE34FFFEC3EF9548F541EE9547F540751B
:103B5200080F200F03023D89AE4AAF4B7C007D0265
:103B6200121EDCD3E53F9FEE6480F8E53E64809848
:103B72004024E54620E5067551007550000551AF19
:103B820051EFD394504003755150E551C3940A400C
:103B92005053080E804BAE4AAF4B7C007D02121E82
:103BA200DCC3E49FFFE49EFEC3E53F9FEE6480F822
:103BB200E53E6480985024E54620E4067551007580
:103BC20050000551AF51EFD394504003755150E569
:103BD20051C3940A400B53080D800675510075506D
:103BE20000AE4AAF4B7C007D02121EDCD3E5419F42
:103BF200EE6480F8E5406480984024E54620E706BC
:103C0200754F00754900054FAF4FEFD394504003F5
:103C1200754F50E54FC3940A405D53080B8058AE70
:103C22004AAF4B7C007D02121EDCC3E49FFFE49E80
:103C3200FEC3E5419FEE6480F8E540648098503110
:103C4200D3E5489400E547648094804024E546200B
:103C5200E606754F00754900054FAF4FEFD39450FC
:103C62004003754F50E54FC3940A400B5308078039
:103C720006754F00754900AF3FAE3E126ED28E42BE
:103C82008F43C374289543FFE49542FEEF7802C345
:103C920033CE33CED8F9FFAD507C00C3EF9DF5454E
:103CA200EE9CF544C3E5446480948050067544005C
:103CB200754500E551C39450501DAF517E007C0004
:103CC2007D7F121ECA7C007D50121EDCEF2480FF15
:103CD200EF64FFF5FA8027C3E5439428E542648048
:103CE20094805017E550C394A050100550C3E5448A
:103CF2006480948040088545FA800375FA00AF41DC
:103D0200AE40126ED28E428F43C374289543FFE4B5
:103D12009542FEEF7802C333CE33CED8F9FFAD49D8
:103D22007C00C3EF9DF545EE9CF544C3E5446480F9
:103D320094805006754400754500E54FC394505079
:103D42001DAF4F7E007C007D7F121ECA7C007D501D
:103D5200121EDCEF2480FFEF64FFF5FE803BC3E51B
:103D6200439428E542648094805017E549C394A0A7
:103D720050100549C3E54464809480401C8545FE8B
:103D8200801775FE008012755100755000754F0046
:103D920075490075FA0075FE00E508C454F0FFEF9E
:073DA200240FF5468546A041
:013DA90022F7
:106E53004310000043D8000044A200004511000085
:106E63004554800045B400004622000046BD0000A2
:106E730000C700C70002000A0E0F03840E0F03842D
:106E830000010001000000000000000000000000FD
:106DB900011400011663011200011700011A00C134
:036DC90013C19261
:030003000265860D
:10658600C0E0C083C08263A201C083C082C0D07550
:10659600D000C006C00720124F20134CD2B330B330
:1065A600020512051AAF1AC3EF64809488401CAF27
:1065B60017EF3395E0FE74402FF58274003EF583A5
:1065C600E512F07512000517751A00E5122512F589
:1065D60012C3E51764809484404F751700D2139058
:1065E6000048E0FF8F12804120123E30133BE51237
:1065F6002512F512A2D792B3051AAF1AC3EF64801B
:106606009488401A0517AF17EF3395E0FE74482FAC
:10661600F58274003EF583E0FF8F12751A00C3E51C
:1066260017648094A04002D212D007D006D0D0D0F2
:0D66360082D08363A201D082D083D0E032F5
:1054B300900048E56EF0A3E56FF0E56B2484FFE50B
:1054C3006A3403FE90004AEEF0A3EFF09001FBE094
:1054D300FEA3E0FF90004CEEF0A3EFF09001F9E0A3
:1054E300FEA3E0FFEF2484FFEE3403FE90004EEEB4
:1054F300F0A3EFF0E50B2484FFE50A3403FE9000EC
:1055030050EEF0A3EFF0900022E0FEA3E0FF900046
:1055130052EEF0A3EFF0900024E0FEA3E0FF900032
:1055230054EEF0A3EFF0900028E0FEA3E0FF90001C
:1055330056EEF0A3EFF0900058E54AF0A3E54BF0E8
:10554300300F0B90005AE4F0A37401F08008900030
:105553005AE4F0A3E4F0900015E0FFEF3395E0FE8A
:1055630090005CEEF0A3EFF0900014E0FFEF3395B2
:10557300E0FE90005EEEF0A3EFF0900013E0FFEF8B
:105583003395E0FE900060EEF0A3EFF0900012E0A0
:10559300FFEF3395E0FE900062EEF0A3EFF0900092
:1055A30011E0FFEF3395E0FE900064EEF0A3EFF01F
:1055B300900041E0F516900040E4F0A37463F0C35B
:1055C300E5166480948840030256A4C3E5166480FC
:1055D300948050030256A4900042E0F518A3E0F52E
:1055E30019AF16EF3395E0FEEF25E0FFEE33FE74BF
:1055F300732FF582746E3EF583E493FE740193FF7B
:10560300D3E5199FEE6480F8E5186480984021AFD4
:1056130016EF3395E0FEEF25E0FFEE33FE74732FB4
:10562300F582746E3EF583E493F518740193F519CE
:10563300AF16EF3395E0FEEF25E0FFEE33FE748304
:105643002FF582746E3EF583E493FE740193FFC3DA
:10565300E5199FEE6480F8E5186480985021AF1631
:10566300EF3395E0FEEF25E0FFEE33FE74832FF575
:1056730082746E3EF583E493F518740193F519AFC4
:1056830016EF3395E0FEEF25E0FFEE33FE74222F95
:10569300F58274003EF583E518F0A3E519F0125185
:0C56A3003EE516B40805A20FB3920F22DA
:03002B000264C4A8
:1064C400C0E0C0F0C083C08263A201C083C082C0A8
:1064D400D075D000C000C001C002C003C004C00514
:1064E400C006C00775A61E75A6E11509AF09EF70B1
:1064F4006D75090453907790003AE0FEA3E0FFEF36
:106504008EF01220AB6531000065360001653B005A
:10651400026540000365450004654A0005654F00B7
:106524000665540007655900080000655C1268EFB1
:106534008026126ACB8021126C8B801C1262ED8043
:106544001712000E8012125DCC800D125EE48008DA
:10655400125FF880031258614390881238B2C2CF98
:10656400D007D006D005D004D003D002D001D0008B
:10657400D0D0D082D08363A201D082D083D0F0D097
:02658400E03203
:03002300026D1B50
:106D1B00C0E0C0F0C083C08263A201C083C082C048
:106D2B00D075D000C000C001C002C003C004C005B4
:106D3B00C006C007C2AC30981AC298E599B43F039D
:106D4B0012528BE599B4210B1256AFD214D215D235
:106D5B0016D217C299D2ACD007D006D005D004D02A
:106D6B0003D002D001D000D0D0D082D08363A20157
:096D7B00D082D083D0F0D0E032C8
:03000B0002664347
:10664300C0E0C0F0C083C08263A201C083C082C027
:10665300D075D000C000C001C002C003C004C00593
:10666300C006C007758A00758C4C75A61E75A6E119
:106673000514AF14C3EF6480948A40163012137567
:106683001400751700751A00C213C2127512001296
:1066930054B3E51375F007121E50AFF0EF701B12E1
:1066A300422D301804D214D217E57660073018044F
:1066B300D215D21612002E12508F1513AF13EF708E
:1066C3000C75134ED218301804D215D216D007D039
:1066D30006D005D004D003D002D001D000D0D0D052
:0F66E30082D08363A201D082D083D0F0D0E03286
:10224500758FFF758921758DFF438780759850D2ED
:102255008CD28ED2CA75CB4C75CA0043B71143B820
:1022650021D28875D90243D84075DA4275DE42C25B
:10227500187513467509017F02125D16125D6375A7
:102285007700900040E4F0A37463F020A003126B84
:102295006575A8B275A70712514B12516DC20F9003
:1022A500006CE0FEA3E0FFEF4E6004D2108002C296
:1022B50010900068E0F560A3E0F56190006AE0F534
:1022C5005AA3E0F55BE57670FC900036E0FCA3E0F0
:1022D500FDEC121B977B007A0079207841121A7762
:1022E5007B007A00793478C312187D9001E2E0F81A
:1022F500A3E0F9A3E0FAA3E0FB12196E90001E1209
:102305002028900038E0FCA3E0FDEC121B977B0031
:102315007A0079207841121A777B007A0079B478AF
:10232500C212187D9001E2E0F8A3E0F9A3E0FAA358
:10233500E0FB12196E90001A122028900011E0FCA3
:10234500EC121B9C7B007A0079B47844121A77C092
:1023550004C005C006C007900012E0FCEC121B9CEF
:102365007B007A0079C07841121A77A804A905AADA
:1023750006AB07D007D006D005D00412187DC004DF
:10238500C005C006C007900010E0FCEC121B9C7B4A
:10239500007AC079A87847121A77A804A905AA0671
:1023A500AB07D007D006D005D00412187D900044A5
:1023B500122028900014E0FFEF3395E0FEFDFCEFBE
:1023C5002409FFEE3400FEED3400FDEC3400FC7B07
:1023D5000C7A0079007800126DCDA804A905AA062B
:1023E500AB07900015E0FFEF3395E0FEFDFCEF2411
:1023F500D0FFEE3407FEED3400FDEC3400FCEB2F8E
:10240500FFEA3EFEE93DFDE83CFC7B077A007900EA
:102415007800121F287B047A0079007800126DCDB0
:10242500C004C005C006C007900015E0FFEF339556
:10243500E0FEFDFC7B6F7A0179007800121F28D041
:1024450003D002D001D000C3EF9BFFEE9AFEED99B9
:10245500FDEC98FCC004C005C006C007900014E060
:10246500FFEF3395E0FEFDFC7B137A0179007800E0
:10247500121F287B097A0079007800126DCDA80417
:10248500A905AA06AB07D007D006D005D004EB2FC7
:10249500FBEA3EFAE93DF9E83CF8900013E0FFEF6E
:1024A5003395E0FEFDFCEB2FFFEA3EFEE93DFDE83E
:1024B5003CFCEF247AF511EE34E0F510ED3400F52F
:1024C5000FEC3400F50E900028E0FEA3E0FFEF646A
:1024D500014E70487B017A007908C003C002C00133
:1024E5007B017A0079789001ABEBF0A3EAF0A3E9E0
:1024F500F0AF11AE10AD0FAC0E9001AE12202890CA
:102505000044E0FCA3E0FDA3E0FEA3E0FF9001B2E0
:10251500122028D001D002D003124678900028E07E
:10252500FEA3E0FFEF4E60030227BF7B017A00792F
:1025350008C003C002C0017B017A007978900123AD
:10254500EBF0A3EAF0A3E9F0AF11AE10AD0FAC0EBE
:10255500900126122028900044E0FCA3E0FDA3E0B2
:10256500FEA3E0FF90012A122028D001D002D0035B
:10257500122B94AF11AE10AD0FAC0EC004C005C048
:1025850006C007900044E0FCA3E0FDA3E0FEA3E045
:10259500FF90015E122028D007D006D005D0041286
:1025A5000D47A804A905AA06AB077F007E3E7DC698
:1025B5007C481218797B007A00797A7844121A7768
:1025C500A804A905AA06AB077F007EC07D3C7C4513
:1025D500121879C004C005C006C00790001AE0FCB7
:1025E500A3E0FDA3E0FEA3E0FF125A4DA804A90550
:1025F500AA06AB07D007D006D005D00412196EC0C5
:1026050004C005C006C007900016E0FCA3E0FDA3CA
:10261500E0FEA3E0FF125A63A804A905AA06AB07CA
:10262500D007D006D005D00412196EC004C005C06D
:1026350006C007900078E0FCA3E0FDA3E0FEA3E060
:10264500FF125A4DA804A905AA06AB07D007D00664
:10265500D005D00412196EC004C005C006C007AF6E
:1026650011AE10AD0FAC0EC004C005C006C0077F8B
:10267500AB7EAA7D0A7CBF900044E0F8A3E0F9A3F5
:10268500E0FAA3E0FB12187D90015E122028D00726
:10269500D006D005D004120D47C004C005C006C041
:1026A50007AF11AE10AD0FAC0EC004C005C006C01B
:1026B500077F007E007D207CBF900044E0F8A3E00A
:1026C500F9A3E0FAA3E0FB12187D90015E12202821
:1026D500D007D006D005D004120D47D003D002D0C4
:1026E50001D0001218797B337A337993783F121A27
:1026F50077A804A905AA06AB07D007D006D005D050
:102705000412187D121BD08E0C8F0D90003CE0FE3C
:10271500A3E0FFC3EF9404EE64809480504FAC0CAB
:10272500AD0DEC121B97C004C005C006C007900094
:102735003CE0FEA3E0FFEF7802C333CE33CED8F9F9
:10274500FF74532FF582746E3EF583121FF8D00780
:10275500D006D005D00412196E7B007A00797A78FC
:1027650044121A77121BD08E1B8F1C804DAC0CADFA
:102775000DEC121B97C004C005C006C00790003CB5
:10278500E0FEA3E0FFEF7802C333CE33CED8F9FFE6
:1027950074532FF582746E3EF583121FF8D007D05F
:1027A50006D005D00412196E7B007A40791C784654
:1027B500121A77121BD08E1B8F1C900028E0FEA3E7
:1027C500E0FFEF64024E70149000781220343F82CF
:1027D500D0E590000812203440C39DB2900028E057
:1027E500FEA3E0FFEF64034E7014900078122034CE
:1027F5003F3566CF90000812203440A73B64900017
:1028050028E0FEA3E0FFEF64044E701490007812F8
:102815002034BF018FC590000812203440953F7DBC
:10282500900028E0FEA3E0FFEF64054E70149000D1
:10283500781220343EC44D019000081220343FB96F
:102845001687900028E0FEA3E0FFEF64064E7014A3
:102855009000781220343F32B6AE90000812203432
:10286500401F2B02900028E0FEA3E0FFEF64074E17
:1028750070149000781220340000000090000812B7
:10288500203440BC7AE1900028E0FEA3E0FFEF642D
:10289500084E7067900032E0FCA3E0FDEC121B9738
:1028A5007B007A0079207841121A779001E2E0F8EE
:1028B500A3E0F9A3E0FAA3E0FB12196E9000081259
:1028C5002028900034E0FCA3E0FDEC121B977B0070
:1028D5007A0079207841121A777B007A0079B478EA
:1028E500C212187D9001E2E0F8A3E0F9A3E0FAA393
:1028F500E0FB12196E900078122028900028E0FE67
:10290500A3E0FFC3EF9409EE648094804003022A9C
:1029150013900044E0FCA3E0FDA3E0FEA3E0FFC0AC
:1029250004C005C006C007AF11AE10AD0FAC0E90C8
:1029350001CE122028D007D006D005D004124A4077
:102945009001881220287B017A00790CC003C0020F
:10295500C0017B017A007900900185EBF0A3EAF0D4
:10296500A3E9F0900008E0FCA3E0FDA3E0FEA3E0EE
:10297500FF90018C122028900078E0FCA3E0FDA3D5
:10298500E0FEA3E0FF900190122028D001D002D0F4
:102995000312339B900028E0FEA3E0FFEF4E705A30
:1029A500900000E0FCA3E0FDA3E0FEA3E0FF125AC7
:1029B5004D7B007A5079C7784512196EC004C00561
:1029C500C006C0079000E812203448B98C00D00733
:1029D500D006D005D004126A2EA804A905AA06AB14
:1029E50007900000E0FCA3E0FDA3E0FEA3E0FF12DA
:1029F50018799000041220288014900000E0FCA3B0
:102A0500E0FDA3E0FEA3E0FF900004122028900063
:102A150028E0FEA3E0FFEF64094E705C90002EE015
:102A2500FCA3E0FDEC121B977B007A00792078412E
:102A3500121A779001E2E0F8A3E0F9A3E0FAA3E027
:102A4500FB12196E90000C122028900030E0FCA3B8
:102A5500E0FDEC121B977B007A0079207841121A71
:102A6500779001E2E0F8A3E0F9A3E0FAA3E0FB1216
:102A7500196E900004122028900028E0FEA3E0FFC4
:102A8500EF640A4E705C90002AE0FCA3E0FDEC12B6
:102A95001B977B007A0079207841121A779001E222
:102AA500E0F8A3E0F9A3E0FAA3E0FB12196E9000A9
:102AB5000C12202890002CE0FCA3E0FDEC121B97E3
:102AC5007B007A0079207841121A779001E2E0F8CC
:102AD500A3E0F9A3E0FAA3E0FB12196E900004123B
:102AE50020289001E2E0F8A3E0F9A3E0FAA3E0FBD7
:102AF50090000CE0FCA3E0FDA3E0FEA3E0FF121AAA
:102B0500777BCD7ACC794C783D12187D7B007A00A5
:102B15007920784112196E121BD08E6E8F6F90013D
:102B2500E2E0F8A3E0F9A3E0FAA3E0FB900004E0FB
:102B3500FCA3E0FDA3E0FEA3E0FF121A777BCD7AAC
:102B4500CC794C783D12187D7B007A00792078414C
:102B550012196E121BD08E6A8F6B7F007E007D204E
:102B65007C41900078E0F8A3E0F9A3E0FAA3E0FB4C
:102B750012196E9001E2E0F8A3E0F9A3E0FAA3E0F0
:0F2B8500FB121A77121BD08E0A8F0B0222CA2264
:105CAF00EFC0E0C283740F125CE47430125CEE74C8
:105CBF0005125CE47430125CEE7401125CE4743013
:105CCF00125CEE7401125CE4D0E0146002740844BC
:105CDF0020125CFC227D000000DDFCD5E0F7225491
:105CEF00F053800F4280C282D283C28322C282804D
:105CFF0002D282C0E0125D0AD0E0C454F053800F8C
:105D0F004280D283C28322125CAF125D48740612A6
:105D1F005CFC125D48740E125CFC125D487401123B
:105D2F005CFC125D487440125CFC125D95125D487C
:105D3F007480125CFC125D7522740A125CE422EF0F
:105D4F00C0E0125D48D0E0125D0022125D4874027F
:105D5F00125CFC22125D487401125CFC22125D4839
:105D6F00740E125CFC22125D48740C125CFC221241
:105D7F005D48740F125CFC22EFC0E0125D48D0E06A
:105D8F004480125CFC22905DA47E28E493FF125D98
:105D9F004EA3DEF7220004040E0E1F1F00001F1F6C
:105DAF000E0E04040000101C1F1C10000000010741
:0D5DBF001F070100000E11171917110E002B
:106EBA007A107B00EE6BFB8BF053F080ABF033EF74
:086ECA0033FFEE33FEDAEE2285
:106BFA00900207EEF0A3EFF0900207E0FEA3E0FF99
:106C0A007C037DE8121EDCEF2430F5993099FDC231
:106C1A0099900207E0FEA3E0FF7C037DE8121EDCE8
:106C2A007E007F64CFCDCFCECCCE121EDCEF2430D7
:106C3A00F5993099FDC299900207E0FEA3E0FF7C26
:106C4A00007D64121EDC7E007F0ACFCDCFCECCCE73
:106C5A00121EDCEF2430F5993099FDC29990020793
:106C6A00E0FEA3E0FF7C007D0A121EDCAF05EF24E4
:106C7A0030F5993099FDC2997599003099FDC299FC
:016C8A0022E7
:10528B009001FD122034000186A020983E9001FD74
:10529B00E0FCA3E0FDA3E0FEA3E0FFEC4D4E4F606E
:1052AB002A9001FDE0FCA3E0FDA3E0FEA3E0FF7B61
:1052BB00FF7AFF79FF78FFEF2BFFEE3AFEED39FD1A
:1052CB00EC38FC9001FD12202880BFC298AF99EFFB
:1052DB00122085533061533C6253486353506453DF
:1052EB005C65536866537467538068538C69539835
:1052FB006A53A46B53B06C53BC6D53C86E53D66FCB
:10530B0053E27053F67153FE72540C73541A745467
:10531B005F75546D76547B7754897854977954A57F
:10532B007A000054B2900022E0FEA3E0FF126BFA69
:10533B0022900024E0FEA3E0FF126BFA22AF4BAEEB
:10534B004A126BFA22900028E0FEA3E0FF126BFAE0
:10535B002290002AE0FEA3E0FF126BFA2290002CB1
:10536B00E0FEA3E0FF126BFA2290002EE0FEA3E01A
:10537B00FF126BFA22900030E0FEA3E0FF126BFAF3
:10538B0022900032E0FEA3E0FF126BFA2290003471
:10539B00E0FEA3E0FF126BFA22900036E0FEA3E0E2
:1053AB00FF126BFA22900038E0FEA3E0FF126BFABB
:1053BB002290003AE0FEA3E0FF126BFA22E50D24E7
:1053CB0088FFE50C3413FE126BFA229001FBE0FE12
:1053DB00A3E0FF126BFA229001F9E0FEA3E0FFEFCE
:1053EB002484FFEE3403FE126BFA22AF6FAE6E1203
:1053FB006BFA22E56B2484FFE56A3403FE126BFA29
:10540B0022E50B2484FFE50A3403FE126BFA22A279
:10541B000FE433FFEF3395E0FEEFC4F8540FC86889
:10542B00FFEEC454F048FEE5A0C4540FFD7C00EF22
:10543B002DFDEE3CFCA210E433FFEF3395E0FEEFC5
:10544B007805C333CE33CED8F9FFED2FFFEC3EFEFC
:10545B00126BFA22900010E0FFEF3395E0FE126B17
:10546B00FA22900011E0FFEF3395E0FE126BFA2267
:10547B00900012E0FFEF3395E0FE126BFA229000E2
:10548B0013E0FFEF3395E0FE126BFA22900014E06D
:10549B00FFEF3395E0FE126BFA22900015E0FFEF61
:0754AB003395E0FE126BFADD
:0154B20022D7
:10684A009001EEE4F0A3E4F09001F4E4F09001F496
:10685A00E0FFD3EF6480948340030268E69001F07E
:10686A00122034000186A020983E9001F0E0FCA39B
:10687A00E0FDA3E0FEA3E0FFEC4D4E4F602A90013D
:10688A00F0E0FCA3E0FDA3E0FEA3E0FF7BFF7AFFBC
:10689A0079FF78FFEF2BFFEE3AFEED39FDEC38FC7D
:1068AA009001F012202880BFC2989001EEE0FEA36A
:1068BA00E0FF7C007D0A121ECAAD997C00EF2DFF15
:1068CA00EE3CFEEF24D0FFEE34FFFE9001EEEEF038
:1068DA00A3EFF09001F4E004F00268579001EEE0B3
:0468EA00FEA3E0FF2A
:0168EE002287
:1056AF00900201122034000186A020983E90020142
:1056BF00E0FCA3E0FDA3E0FEA3E0FFEC4D4E4F6046
:1056CF002A900201E0FCA3E0FDA3E0FEA3E0FF7B34
:1056DF00FF7AFF79FF78FFEF2BFFEE3AFEED39FDF2
:1056EF00EC38FC90020112202880BFC298AF99EFCE
:1056FF00122085574861575762576663577564572D
:10570F00846557936657A26757B16857C06957CFDB
:10571F006A57DE6B57ED6C57FC6D580B7258107350
:10572F00581374581975582576583177583D78584D
:10573F00497958557A0000586012684A900022EE55
:10574F00F0A3EFF012513E2212684A900024EEF0BF
:10575F00A3EFF012513E2212684A900026EEF0A3FA
:10576F00EFF012513E2212684A900028EEF0A3EF9C
:10577F00F012513E2212684A90002AEEF0A3EFF089
:10578F0012513E2212684A90002CEEF0A3EFF01255
:10579F00513E2212684A90002EEEF0A3EFF0125104
:1057AF003E2212684A900030EEF0A3EFF012513E05
:1057BF002212684A900032EEF0A3EFF012513E220F
:1057CF0012684A900034EEF0A3EFF012513E22120D
:1057DF00684A900036EEF0A3EFF012513E221268A5
:1057EF004A900038EEF0A3EFF012513E2212684AB1
:1057FF0090003AEEF0A3EFF012513E22D20DD211EB
:10580F0022D21122A20FB3920F2212684A900010D7
:10581F00EFF012503A2212684A900011EFF0125036
:10582F003A2212684A900012EFF012503A22126890
:10583F004A900013EFF012503A2212684A90001467
:10584F00EFF012503A2212684A900015EFF0125002
:01585F003A0E
:015860002225
:10187600021C3CE86480F8E933E83360110460F048
:10188600ED33EC337009E8FCE9FDEAFEEBFF2204D8
:1018960060DED3EB9FEA9EE99DE8C2E78CF0C2F7D3
:1018A60095F0400CE8CCF8E9CDF9EACEFAEBCFFB9F
:1018B600121C0785D0F05804700320D5B3E80470D5
:1018C600075002B2D5021C4692D5EC0460F7E4CC70
:1018D600C0E0C398F8603B94186008400DD0E0FB68
:1018E600021C1EE4FBFAC9FC8028E830E406E4C9C1
:1018F600FBE4CAFCE830E305E4C9CACBFCE85407BC
:101906006010F8C3E913F9EA13FAEB13FBEC13FCC6
:10191600D8F130F52FC3E49CFCEF9BFFEE9AFEED69
:1019260099FDD0E0FBEF4E4D4C701222DB03021CFA
:1019360043EC2CFCEF33FFEE33FEED33FDED30E7E9
:10194600EB021C1EEF2BFFEE3AFEED39FDD0E0FB5D
:1019560050130BBB0003021C46ED13FDEE13FEEF06
:0819660013FFEC13FC021C1E30
:10196E00EC4D6011E8497017ED33EC3304600DE473
:10197E00FCFFFEFD22E933E8330470F8021C3C1232
:10198E001C0758046009E4CC248150062850090233
:10199E001C46284003021C43C0E0EB4A7044B98049
:1019AE0006D0E0FB021C32EF4E701CBD8008EBFF30
:1019BE00EAFEE9FD80EBE98DF0A4FEE5F0021A5790
:1019CE00E9CDF9EAFEEBFFEF89F0A4FCE5F0CE8954
:1019DE00F0A42EFFE435F0CD89F0A42DFEE435F011
:1019EE008067EF4E7005BD80D780C3EF8BF0A4AC3F
:1019FE00F0EE8BF0A42CFCE435F0F8EF8AF0A42C7A
:101A0E00E5F038FCE433CB8DF0A42CFCE5F03BF88C
:101A1E00EE8AF0A42CFCE5F038F8E433CF89F0A47C
:101A2E002CFCE5F038CF3400CE89F0A42FFFE5F082
:101A3E003EFEE433C98DF0A42EFEE5F039CD8AF0DA
:101A4E00A42FFFE5F03EFEE43DFD33D0E0FB500752
:101A5E000BBB000F021C46EC2CFCEF33FFEE33FEEB
:061A6E00ED33FD021C1E19
:101A7400021C46EC5D046005E859047003021C3C3A
:101A8400121C07580460F6EC4860F2EC7004FDFE8A
:101A9400FF22C860DB2481C85009C3986002500645
:101AA400021C439850CAF582E9294B4A7005AB825F
:101AB400021C3275F0007C1A7880C3EF9BEE9AED1D
:101AC40099400DC3EF9BFFEE9AFEED99FDE842F0BD
:101AD400DC23ACF0D0E0FFD0E0FED0E0FDAB822010
:101AE400E7101BEB60BAEC2CFCEF33FFEE33FEED9A
:101AF40033FD021C1EE803F830E705C0F075F00062
:101B0400EF2FFFEE33FEED33FD40B830E7C280AA7D
:101B140074F8CC6480CCC86480C8F582046043C384
:101B2400EB9FF5F0EA9E42F0E99D42F0E89C45F017
:101B340060305018E5825FFFE582F42B5582FB503C
:101B4400210ABA001D09B90019088016E5825BFB59
:101B5400E582F42F5582FF50090EBE00050DBD002D
:101B6400010CC3EB9FF5F0EA9E42F0E99D42F0E8D8
:0D1B74009C45F06007CC4820E701B3EC224F
:101B8100ED33EC33600A047003BD8004ECB2E7FC72
:011B91002231
:101B920075F020800E75F010800575F0087D007ECE
:101BA200007F003392D530D503121F77EC334010FB
:101BB200EF33FFEE33FEED33FDEC33FCD5F0ED22D7
:0E1BC200E5F0247EA2D513CC92E7CDCEFF2213
:101BD000EDD2E7CD33EC3392D524814006E4FFFE0D
:101BE000FDFC22FCE4CFCECDCC24E0501174FF806C
:101BF000EDC3CC13CCCD13CDCE13CECF13CF047009
:071C0000F030D5DE021F7772
:103DAA00E57B24F3F582E43400F583E0057B229079
:103DBA0000F03009039000F3E475F0011220650267
:103DCA001E722002E97F2ED2028018EF540F24902F
:103DDA00D43440D4FF30060BEF24BFB41A0050038A
:103DEA002461FFE57C6002157C057FE57F70020592
:103DFA007E30090E9000F0E475F001122065EF02A2
:103E0A001EB8026E937403D2098003E4C209F57BDB
:103E1A009000F012207CE4F57CF57EF57FE57C606D
:103E2A00077F20123DED80F5757DFFC203C202C2F5
:103E3A0004C205C207C208C20A123DB9FF700D309A
:103E4A0009057F00123DFEAF7FAE7E22B4255FC218
:103E5A00D5C206123DB9FF24D0B40A00501A75F033
:103E6A000A787C30D50508B6FF0106C6A426F620D6
:103E7A00D5047002D20580D924CFB41A00EF5004B9
:103E8A00C2E5D2060240F0D20380C6D20280C0D276
:103E9A000480BCD2D580BAD20780B47F20123DED0F
:103EAA002004077401B57C0040F1123DAAFF123DBF
:103EBA00ED023E27D20AD2088095123DAAFB123D96
:103ECA00AAFA123DAAF94A4B700679EE7A417BFFAB
:103EDA0020042EE57C602A7E008E82758300121EE5
:103EEA008B60060EEE657D70F0C2D5EBC0E0EAC0CD
:103EFA00E0E9C0E0EE124151D0E0F9D0E0FAD0E0BA
:103F0A00FB121E72FF60AAEBC0E0EAC0E0E9C0E063
:103F1A00123DEDD0E02401F9D0E03400FAD0E0FB04
:103F2A00E57D0460DCD57DD98087D20480A2124168
:103F3A003360F7E57D700104121C51A97D600DE51F
:103F4A007D600914F57D1241DBEF60F3EA30E70288
:103F5A00F404C3995079EAF4257D0430E701E404B6
:103F6A00F57D800D12413360C1EA057D257D121C65
:103F7A0051EA90011FF030E701E4257D04D57D0464
:103F8A0020070114124151E4C0E01241DB90011FE5
:103F9A00E0601320E70714F0123DD5802204F0D028
:103FAA00E014C0E07F00123DD5E57D6007123DCCEC
:103FBA00157D800B300703123DCCD0E0023E27D09E
:103FCA00E00480C4124133609EE57D04121C5190C6
:103FDA00011FEAF0E57D2007026001042404124172
:013FEA005185
:103FEB0074FF04C0E01241DB123DD5E57D200702D2
:103FFB006003123DCCD0E0B57DE87F45123DDF90EC
:10400B00011FE07F2B30E7047F2DF404C0E0123D4D
:10401B00EDD0E075F00A84C0F0123DD6D0E0123D31
:10402B00D6023E27791080027908C208C20A80089E
:10403B00D2D5790A8004790AC2D5E57D047002F5E0
:10404B007DE4FAFDFEFF123DAAFC7B082003131250
:10405B003DAAFD7B1030020A123DAAFE123DAAFFBB
:10406B007B20EC3382D592D55013C3E43002069FEC
:10407B00FFE49EFEE42003039DFDE49CFCE4CBF8EF
:10408B00C203EC700CCFCECDCCE824F8F870F380E3
:10409B0017C3EF33FFEE33FEED33FDEC33FCEB33A5
:1040AB00FB994002FB0FD8E9EB300305F8D0E0C4D5
:1040BB0048B203C0E00AEC4D4E4F78207B0070C233
:1040CB00EAB57D0040BCC0E0124153D0F0D0E020F7
:1040DB000304C4C0E0C4B203C0F0123DD6D0F0D587
:1040EB00F0EB023E271220853EC453402F583E95DD
:1040FB004C3E914240334F403B44403B493EAA43E8
:10410B004041553F6E463FCE453F3847420E503EED
:10411B00992D3E9D2E3EC02B3EA1233EBE2041F746
:10412B002A3E594800003EB8E57DB4FF03757D0675
:10413B00123DAAFC123DAAFD123DAAFE123DAAFF9A
:10414B00900118021C8E790AA2D52005143007099C
:10415B00B910020404B9080104A2D52008025001C9
:10416B00042004689204B57C005034C0E07F2030FA
:10417B0005197F30A20472087207500F1241AAC2B0
:10418B0004C208C207C20A7F30800F300703E9C0A0
:10419B00E0123DED300703D0E0F9D0E0B57CCC3038
:1041AB0007177F30B9100C123DED7F583006077F93
:1041BB00788003B90803123DED3004057F2D023DD5
:1041CB00ED7F20200AF87F2B2008F322920480CF6A
:1041DB007F00B40700500B2418F582E43401F583FB
:1041EB00E0FF22286E756C6C2900D203123DAA30B9
:1041FB0003F8C203787C30D50108F6023E592D50E6
:10420B00434958123DAA2403B405004001E49042EF
:10421B000993123DDE743A123DDED205757C040221
:02422B00402F22
:0D6F3900ED33EC3360065004EC6480FC2264
:10679E00021C3C22EDA2E7D2E7F9EC3340F260F3A3
:1067AE00B4FF08ED547F70E8021C46F82481C2E065
:1067BE00C0E0F40428FAC313FCED92E7FD9000E468
:1067CE00122028EEA2E7E9BA7F02C3133400940028
:1067DE00FA75F091A4E5F013F494FE8AF0A433E573
:1067EE00F033248CD313FDE492E7FE7F007C3F75DB
:1067FE008302ECC0E0F8EDC0E0F9EEC0E0FAEFC0C5
:10680E00E0FB8583F09000E4121FD085F083121A0E
:10681E0077D0E0FBD0E0FAD0E0F9D0E0F812187DA6
:10682E00ED6480FD30E7011CD583C7ED33CC33F822
:0C683E00D0E0A2E71328C313CC13FD2206
:106A2E009000E41220289000E8E0F8A3E0F9A3E03B
:106A3E00FAA3E0FB9000E4E0FCA3E0FDA3E0FEA3DC
:106A4E00E0FF121A77125BAD9000E412202890003E
:106A5E00E8E030E7599000E4E0FCA3E0FDA3E0FE9F
:106A6E00A3E0FFECC0E0EDC0E0EEC0E0EFC0E0E47C
:106A7E00FFFEFDFC9000E4E0F8A3E0F9A3E0FAA32A
:106A8E00E0FB121B147BDB600250087A0F79497809
:106A9E004080067A0F794978C0D0E0FFD0E0FED072
:106AAE00E0FDD0E0FC12187D9000E412202890004A
:0D6ABE00E4E0FCA3E0FDA3E0FEA3E0FF2266
:105A05003A70FA83BCAAE9E43E81E0F8BF9DE9E675
:105A15003F80000039283C1ABB9969663DA335E3F0
:105A2500BF255DE73FC90FDB418DDBCCC44936EEB1
:105A350045C9913FC5B0F83D3F800000C317F53417
:105A4500452FFA73C60AFDDD125B0E04A2E1920032
:105A55001420E015905A057404121D938030125BD2
:105A65000E30E102B20020E0EBA883A9829000E4A9
:105A750012202889828883905A197404121D9385EF
:105A850082F09000E4121FEC85F08212196EED4C45
:105A95006007300004EC6480FC22125B0EC0E0A8B5
:105AA50083A9829000E412202889828883905A3D38
:105AB5007403121D938582F09000E4121FEC85F0AB
:105AC5008212196E9000E4E0CCF0A3E0CDF0A3E0E3
:105AD500CEF0A3E0CFF0905A2D7403121D93D0821F
:105AE5008582F09000E4121FEC85F082E58230E0BB
:105AF50007121A77B2008096EFCBFFEECAFEEDC90A
:105B0500FDECC8FC121A778085ED33EC547FCC335D
:105B1500920024605007D0E0D0E0021C3C7B837AE1
:105B2500F97922783E12196EEDF933ECF8332481B8
:105B35005011EFFBEEFA121BD0121B92ECB2E7FCF0
:105B450012187DED33EC33602F2403F8C313FCEDFD
:105B550092E7FDE82481E4501FECF8EDF9EEFAEF49
:105B6500FB121BD0EF04C2E0FCF582121B9CECB2C9
:105B7500E7FC12187DE58203FAED33EC3360071478
:085B850013FCED92E7FDEA229A
:105B8D00BE1249253E4CCCCDBEAAAAAB3F8000002B
:105B9D003E7ADBB03EED63383F24BC7D3F490FDBE1
:105BAD00ED33ECC2E7CC339200B4FF13ED547F60BC
:105BBD0003021C3C7FDB7E0F7DC97C3F025CA2C2D1
:105BCD0001C3947F401E7007EDD2E794904015EF0E
:105BDD00FBEEFAEDF9ECF87F007E007D807C3F1244
:105BED001A77D201ED33EC33248430E705E4C0E0BD
:105BFD00806B04FAEDD2E754F0C333DAFD54073469
:105C0D00002323C0E0CCC0E0F8EDC0E0F9EEC0E029
:105C1D00FAEFC0E0FBE4121B9CEC24FEFC9000ECC0
:105C2D0012202812196E7B007A007980783F1218A5
:105C3D007D9000ECE0B2E7CCF0A3E0CDF0A3E0CE98
:105C4D00F0A3E0CFF0D0E0FBD0E0FAD0E0F9D0E067
:105C5D00F812187D9000EC121FEC121A779000ECE0
:105C6D00122028905B8D7403121D939000EC121F6F
:105C7D00EC12196ED0E0600F2499F582E4345BF5D7
:105C8D0083121FF812187D30010B7BDB7A0F79C957
:105C9D0078BF12187DED33EC336006ECA20092E76D
:025CAD00FC22D7
:1061FD009000E412202874FFFFFEFDFC9000E4E007
:10620D00F8A3E0F9A3E0FAA3E0FBC3121F85603801
:10621D007F807E967D187C4B9000E4E0F8A3E0F93A
:10622D00A3E0FAA3E0FB121B146002501B7F807EDB
:10623D00967D187CCB9000E4E0F8A3E0F9A3E0FA9A
:10624D00A3E0FB121B14500F9000E4E0FCA3E0FD53
:10625D00A3E0FEA3E0FF229000E4E0FCA3E0FDA399
:10626D00E0FEA3E0FF121BD09000E8122028900062
:10627D00E8E0FCA3E0FDA3E0FEA3E0FFEC121B921F
:10628D00C8ECC8C9EDC9CAEECACBEFCB9000E4E0AB
:10629D00FCA3E0FDA3E0FEA3E0FF121879E4FBFAF6
:1062AD00F9F8121B14602640249000E8E0FCA3E0EE
:1062BD00FDA3E0FEA3E0FFEF24FFFFEE34FFFEEDB4
:1062CD0034FFFDEC34FFFC9000E81220289000E82C
:1062DD00E0FCA3E0FDA3E0FEA3E0FFEC121B922285
:101C0700E9D2E7C933E833F892D5EDD2E7CD33EC23
:071C170033FC5002B2D5229C
:101C1E00EC30E7100FBF000C0EBE00080DBD000427
:101C2E000BEB6014A2D5EB13FCED92E7FD2274FFD3
:101C3E00FCFDFEFF22E480F8A2D574FF13FC7D802C
:031C4E00E480EF40
:101C5100F920E73624F950037907E4F42402FBE57F
:101C610082158270021583DBF6E024FB501BE960CC
:101C710014E4F0E582158270021583E004F0B40AE1
:0D1C810008E4F0D9EE7401F00A22C2D52269
:101C8E00ED33EC3392D5FA602AB4FF33EDC2E77B25
:101C9E00FF60067A1C79B3E4227A1C79BC20D50445
:101CAE007A1C79B7224E614E002B494E46002D49C3
:101CBE004E4600E47A08F0A3DAFC7B00740722C0DB
:101CCE0083C082ECC0E0EDC0E0EEC0E0EFC0E0EA21
:101CDE0075F010A4CAABF075F04DA42BFBE435F0F3
:101CEE00FCEA2410FAEB34C5FBEC34D9FCEDC2E768
:101CFE00FF75F056A4F42411C5F0F434C58FF0A48A
:101D0E002AE5F03BE43CF020E714121E10D0E0FF71
:101D1E00D0E0FED0E0FDD0E0FC121A778014F4047F
:101D2E00121E10D0E0FFD0E0FED0E0FDD0E0FC129D
:101D3E00196ED082D083E0FAEDD2E7CD33EC3324A6
:101D4E0082FBE4C3CF33CFCE33CECD33CD33DBF3F3
:101D5E007B0775F00A846004F0A31B0AE5F0F0A37C
:101D6E008FF0740AA4FFACF08EF0740AA42CFEACB3
:101D7E00F050010C8DF0740AA42CFDE435F0F0A3A4
:051D8E00DBDE740722FA
:101D9300C0E0EFFBEEFAEDF9ECF812196ED0E0F5C6
:101DA300F0EFFBEEFAEDF9ECF8121FDCA3A3A3A30B
:101DB300E8C0E0E9C0E0EAC0E0EBC0E0C0F012191F
:101DC3006E121FF8A3A3A3A312187DD0F0D0E0FBDB
:0D1DD300D0E0FAD0E0F9D0E0F8D5F0D4224D
:101DE0003F8000004120000042C80000447A00000B
:101DF000461C400047C35000497424004B1896808D
:101E00004CBEBC205A0E1BCA6753C21C749DC5AE83
:101E1000FB60065407601C2323121E3EEB543860FF
:101E200009121E2A121E3912196EECF8EDF9EEFA9B
:101E3000EFCB22EB121E3980F1543803241C901D85
:101E4000E0FE93FC0EEE93FD0EEE930ECE93FF227A
:1069AE00022245E493A3F8E493A34003F68001F298
:1069BE0008DFF48029E493A3F85407240CC8C333EA
:1069CE00C4540F4420C8834004F456800146F6DFB9
:1069DE00E4800B0102040810204080906D84E47E58
:1069EE00019360BCA3FF543F30E509541FFEE493AE
:1069FE00A360010ECF54C025E060A840B8E493A375
:106A0E00FAE493A3F8E493A3C8C582C8CAC583CA9F
:106A1E00F0A3C8C582C8CAC583CADFE9DEE780BE57
:016DCC0000C6
:101E5000C2D530F707B2D563F0FF05F030E70CB21A
:101E6000D5F4048463F0FF05F080018430D502F4DA
:021E700004224A
:101E7200BB010689828A83E0225002E722BBFE026E
:091E8200E32289828A83E49322A1
:101E8B00BB010CE58229F582E5833AF583E022500C
:101E9B0006E92582F8E622BBFE06E92582F8E22256
:0D1EAB00E58229F582E5833AF583E4932270
:101EB800BB010689828A83F0225002F722BBFE0109
:021EC800F32203
:101ECA00EF8DF0A4A8F0CF8CF0A428CE8DF0A42E2C
:021EDA00FE22E6
:101EDC00C2D5EC30E709B2D5E4C39DFDE49CFCEE21
:101EEC0030E715B2D5E4C39FFFE49EFE1220D8C3A1
:101EFC00E49DFDE49CFC80031220D830D507C3E49C
:061F0C009FFFE49EFE228F
:101F1200C5F0F8A3E028F0C5F0F8E582158270025A
:061F22001583E038F022F7
:101F2800E88FF0A4CC8BF0A42CFCE98EF0A42CFC58
:101F38008AF0EDA42CFCEA8EF0A4CDA8F08BF0A4D6
:101F48002DCC3825F0FDE98FF0A42CCD35F0FCEB35
:101F58008EF0A4FEA9F0EB8FF0A4CFC5F02ECD39FA
:0F1F6800FEE43CFCEAA42DCE35F0FDE43CFC2267
:106DCD00C2D5E830E70FB2D5E4C39BFBE49AFAE4F1
:106DDD0099F9E498F8EC30E717B2D5126E03122149
:106DED0069E4C39BFBE49AFAE499F9E498F880030B
:106DFD0012216930D50DE4C39FFFE49EFEE49DFD95
:046E0D00E49CFC22E3
:0E1F7700C3E49FFFE49EFEE49DFDE49CFC227B
:101F8500EB9FF5F0EA9E42F0E99D42F0E89C45F0B2
:011F95002229
:101F9600BB010789828A83021FD05005E9F8022116
:101FA600FBBBFE05E9F802220789828A83021FDC51
:101FB600BB010789828A830220285005E9F802229C
:0A1FC6002DBBFE05E9F802223922C6
:0C1FD000E0FCA3E0FDA3E0FEA3E0FF2284
:101FDC00E493FC740193FD740293FE740393FF224B
:0C1FEC00E0F8A3E0F9A3E0FAA3E0FB2278
:101FF800E493F8740193F9740293FA740393FB223F
:10200800BB010789828A83021FEC5005E9F8022286
:1020180013BBFE05E9F802222089828A83021FF891
:0C202800ECF0A3EDF0A3EEF0A3EFF0222B
:10203400A8828583F0D083D08212204B12204B12C9
:10204400204B12204BE473E493A3C583C5F0C583EE
:10205400C8C582C8F0A3C583C5F0C583C8C582C8F6
:012064002259
:10206500F8E0FBA3A3E0F925F0F0E5821582700204
:072075001583E0FA38F022A8
:09207C00EBF0A3EAF0A3E9F02265
:10208500D083D082F8E4937012740193700DA3A3EA
:1020950093F8740193F5828883E4737402936860FE
:0620A500EFA3A3A380DFFE
:1020AB00D083D082F8E4937012740193700DA3A3C4
:1020BB0093F8740193F5828883E473740293B5F0FB
:0D20CB00067403936860E9A3A3A3A380D863
:106E9300EFB40A07740D126E9E740A309811A89904
:106EA300B8130CC2983098FDA899C298B811F6305F
:076EB30099FDC299F5992237
:106ED200C3EE6480948040028007C3E49FFFE49E77
:026EE200FE228E
:1020D800BC000BBE0029EF8DF084FFADF022E4CCEC
:1020E800F875F008EF2FFFEE33FEEC33FCEE9DECB5
:1020F800984005FCEE9DFE0FD5F0E9E4CEFD22EDFB
:10210800F8F5F0EE8420D21CFEADF075F008EF2F44
:10211800FFED33FD4007985006D5F0F222C398FD35
:052128000FD5F0EA22D2
:10212D0075F008758200EF2FFFEE33FECD33CDCC69
:10213D0033CCC58233C5829BED9AEC99E5829840EC
:10214D000CF582EE9BFEED9AFDEC99FC0FD5F0D6C9
:10215D00E4CEFBE4CDFAE4CCF9A88222B800C1B9F3
:10216D000059BA002DEC8BF084CFCECDFCE5F0CB31
:10217D00F97818EF2FFFEE33FEED33FDEC33FCEB6A
:10218D0033FB10D703994004EB99FB0FD8E5E4F925
:10219D00FA227818EF2FFFEE33FEED33FDEC33FC12
:1021AD00C933C910D7059BE99A4007EC9BFCE99A06
:1021BD00F90FD8E0E4C9FAE4CCFB2275F010EF2F4B
:1021CD00FFEE33FEED33FDCC33CCC833C810D7074B
:1021DD009BEC9AE899400AED9BFDEC9AFCE899F886
:0E21ED000FD5F0DAE4CDFBE4CCFAE4C8F92219
:0C21FB00E6FC08E6FD08E6FE08E6FF2210
:0C220700E2FC08E2FD08E2FE08E2FF2213
:0D221300E6FB08E6F908E6FA08E6CBF8223B
:0D222000E2FB08E2F908E2FA08E2CBF8223E
:0C222D00ECF608EDF608EEF608EFF622DD
:0C223900ECF208EDF208EEF208EFF222E1
:00000001FF
